******************************************************************************
             TMS320C2000 Linker PC v16.9.1                     
******************************************************************************
>> Linked Wed Mar 08 16:04:14 2017

OUTPUT FILE NAME:   <E:/28075_INV/28075 and 28234/INV_V000B000D008_6.1.0_2/Project/../Output/28075 INV.out>
ENTRY POINT SYMBOL: "_c_int00"  address: 0009519c


MEMORY CONFIGURATION

         name            origin    length      used     unused   attr    fill
----------------------  --------  ---------  --------  --------  ----  --------
PAGE 0:
  RAMM0                 00000122   000002de  00000000  000002de  RWIX
  RAMLS0_0              00008000   00000300  00000100  00000200  RWIX
  RAMLS0_1              00008300   00000500  00000000  00000500  RWIX
  RAMLS12345            00008800   00002800  00000000  00002800  RWIX
  RAMD0                 0000b000   00000050  00000028  00000028  RWIX
  RAMD01                0000b050   00000fb0  000005d9  000009d7  RWIX
  RAMGS4567             0000f000   00004000  00002b40  000014c0  RWIX
  BEGIN                 00080000   00000002  00000002  00000000  RWIX
  FLASHACONST           00080002   00000ffe  00000200  00000dfe  RWIX
  FLASHAB               00081000   00003000  00000243  00002dbd  RWIX
  FLASHCTON             00084000   0003c000  00013ab8  00028548  RWIX
  RESET                 003fffc0   00000002  00000000  00000002  RWIX

PAGE 1:
  BOOT_RSVD             00000002   00000120  00000000  00000120  RWIX
  RAMM1                 00000400   00000400  00000200  00000200  RWIX
  ADCA_RESULT           00000b00   00000020  00000018  00000008  RWIX
  ADCB_RESULT           00000b20   00000020  00000018  00000008  RWIX
  ADCD_RESULT           00000b60   00000020  00000018  00000008  RWIX
  CPU_TIMER0            00000c00   00000008  00000008  00000000  RWIX
  CPU_TIMER1            00000c08   00000008  00000008  00000000  RWIX
  CPU_TIMER2            00000c10   00000008  00000008  00000000  RWIX
  PIE_CTRL              00000ce0   00000020  0000001a  00000006  RWIX
  PIE_VECT              00000d00   00000200  000001c0  00000040  RWIX
  DMA                   00001000   00000200  000000e0  00000120  RWIX
  CLA1                  00001400   00000040  0000003e  00000002  RWIX
  CLA1_MSGRAMLOW        00001480   00000080  00000000  00000080  RWIX
  CLA1_MSGRAMHIGH       00001500   00000080  00000000  00000080  RWIX
  EPWM1                 00004000   00000100  00000100  00000000  RWIX
  EPWM2                 00004100   00000100  00000100  00000000  RWIX
  EPWM3                 00004200   00000100  00000100  00000000  RWIX
  EPWM4                 00004300   00000100  00000100  00000000  RWIX
  EPWM5                 00004400   00000100  00000100  00000000  RWIX
  EPWM6                 00004500   00000100  00000100  00000000  RWIX
  EPWM7                 00004600   00000100  00000100  00000000  RWIX
  EPWM8                 00004700   00000100  00000100  00000000  RWIX
  EPWM9                 00004800   00000100  00000100  00000000  RWIX
  EPWM10                00004900   00000100  00000100  00000000  RWIX
  EPWM11                00004a00   00000100  00000100  00000000  RWIX
  EPWM12                00004b00   00000100  00000100  00000000  RWIX
  ECAP1                 00005000   00000020  00000020  00000000  RWIX
  ECAP2                 00005020   00000020  00000020  00000000  RWIX
  ECAP3                 00005040   00000020  00000020  00000000  RWIX
  ECAP4                 00005060   00000020  00000020  00000000  RWIX
  ECAP5                 00005080   00000020  00000020  00000000  RWIX
  ECAP6                 000050a0   00000020  00000020  00000000  RWIX
  EQEP1                 00005100   00000040  00000022  0000001e  RWIX
  EQEP2                 00005140   00000040  00000022  0000001e  RWIX
  EQEP3                 00005180   00000040  00000022  0000001e  RWIX
  DACA                  00005c00   00000010  00000008  00000008  RWIX
  DACB                  00005c10   00000010  00000008  00000008  RWIX
  DACC                  00005c20   00000010  00000008  00000008  RWIX
  CMPSS1                00005c80   00000020  00000020  00000000  RWIX
  CMPSS2                00005ca0   00000020  00000020  00000000  RWIX
  CMPSS3                00005cc0   00000020  00000020  00000000  RWIX
  CMPSS4                00005ce0   00000020  00000020  00000000  RWIX
  CMPSS5                00005d00   00000020  00000020  00000000  RWIX
  CMPSS6                00005d20   00000020  00000020  00000000  RWIX
  CMPSS7                00005d40   00000020  00000020  00000000  RWIX
  CMPSS8                00005d60   00000020  00000020  00000000  RWIX
  SDFM1                 00005e00   00000080  00000080  00000000  RWIX
  SDFM2                 00005e80   00000080  00000080  00000000  RWIX
  MCBSPA                00006000   00000040  00000024  0000001c  RWIX
  MCBSPB                00006040   00000040  00000024  0000001c  RWIX
  SPIA                  00006100   00000010  00000010  00000000  RWIX
  SPIB                  00006110   00000010  00000010  00000000  RWIX
  SPIC                  00006120   00000010  00000010  00000000  RWIX
  SPID                  00006130   00000010  00000000  00000010  RWIX
  WD                    00007000   00000040  0000002b  00000015  RWIX
  NMIINTRUPT            00007060   00000010  00000007  00000009  RWIX
  XINT                  00007070   00000010  0000000b  00000005  RWIX
  SCIA                  00007200   00000010  00000010  00000000  RWIX
  SCIB                  00007210   00000010  00000010  00000000  RWIX
  SCIC                  00007220   00000010  00000010  00000000  RWIX
  SCID                  00007230   00000010  00000010  00000000  RWIX
  I2CA                  00007300   00000040  00000022  0000001e  RWIX
  I2CB                  00007340   00000040  00000022  0000001e  RWIX
  ADCA                  00007400   00000080  00000080  00000000  RWIX
  ADCB                  00007480   00000080  00000080  00000000  RWIX
  ADCD                  00007580   00000080  00000080  00000000  RWIX
  INPUT_XBAR            00007900   00000020  00000020  00000000  RWIX
  XBAR                  00007920   00000020  00000020  00000000  RWIX
  SYNC_SOC              00007940   00000010  00000006  0000000a  RWIX
  DMACLASRCSEL          00007980   00000040  0000001a  00000026  RWIX
  EPWM_XBAR             00007a00   00000040  00000040  00000000  RWIX
  CLB_XBAR              00007a40   00000040  00000000  00000040  RWIX
  OUTPUT_XBAR           00007a80   00000040  00000040  00000000  RWIX
  GPIOCTRL              00007c00   00000180  00000180  00000000  RWIX
  GPIODAT               00007f00   00000030  00000030  00000000  RWIX
  CRAZYDSPRAM           0000bffc   00000004  00000000  00000004  RWIX
  RAMGS012              0000c000   00002800  00001ac4  00000d3c  RWIX
  RAMGS3                0000e800   00000800  00000400  00000400  RWIX
  RAMFLASHDATA          00012000   00000f00  00000c60  000002a0  RWIX
  RAMEEPROMDATA         00012f00   00000100  00000082  0000007e  RWIX
  EMIF1                 00047000   00000800  00000070  00000790  RWIX
  DEV_CFG               0005d000   00000180  0000012e  00000052  RWIX
  ANALOG_SUBSYS         0005d180   00000080  00000048  00000038  RWIX
  CLK_CFG               0005d200   00000100  00000032  000000ce  RWIX
  CPU_SYS               0005d300   00000100  00000082  0000007e  RWIX
  ROMPREFETCH           0005e608   00000002  00000002  00000000  RWIX
  DCSM_Z1               0005f000   00000030  00000024  0000000c  RWIX
  DCSM_Z2               0005f040   00000030  00000024  0000000c  RWIX
  DCSM_COMMON           0005f070   00000010  00000008  00000008  RWIX
  MEMCFG                0005f400   00000080  00000080  00000000  RWIX
  EMIF1CONFIG           0005f480   00000020  00000020  00000000  RWIX
  ACCESSPROTECTION      0005f4c0   00000040  00000040  00000000  RWIX
  MEMORYERROR           0005f500   00000040  00000040  00000000  RWIX
  ROMWAITSTATE          0005f540   00000002  00000002  00000000  RWIX
  FLASH0_CTRL           0005f800   00000300  00000182  0000017e  RWIX
  FLASH0_ECC            0005fb00   00000040  00000028  00000018  RWIX
  DCSM_Z1_OTP           00078000   00000020  00000020  00000000  RWIX
  DCSM_Z2_OTP           00078200   00000020  00000020  00000000  RWIX


SECTION ALLOCATION MAP

 output                                  attributes/
section   page    origin      length       input sections
--------  ----  ----------  ----------   ----------------
CLAscratch 
*          0    00008000    00000100     UNINITIALIZED
                  00008000    00000100     --HOLE--

.const_cla 
*          0    00008300    00000000     UNINITIALIZED

Cla1Prog   0    00008800    00000000     UNINITIALIZED

codestart 
*          0    00080000    00000002     
                  00080000    00000002     F2807x_CodeStartBranch.obj (codestart)

.FlashAconst 
*          0    00080002    00000200     
                  00080002    00000200     MainProcedure.obj (.FlashAconst)

Flash28_API 
*          0    00081000    00000243     RUN ADDR = 0000b050
                  00081000    00000243     MainProcedure.obj (Flash28_API)

.CriticalIntFuncsNOTSecured 
*          0    00084000    00002b40     RUN ADDR = 0000f000
                  00084000    00002b40     MainProcedure.obj (.CriticalIntFuncsNOTSecured)

.text      0    00086b40    0000e84f     
                  00086b40    0000ded2     MainProcedure.obj (.text)
                  00094a12    000003d9     MainProcedure.obj (.text:retain)
                  00094deb    000001cd     rts2800_ml.lib : memory.obj (.text)
                  00094fb8    00000107                    : ll_div28.obj (.text)
                  000950bf    00000083                    : fs_div28.obj (.text)
                  00095142    0000005a                    : fs_mpy28.obj (.text)
                  0009519c    00000054                    : boot28.obj (.text)
                  000951f0    0000002a                    : l_div28.obj (.text)
                  0009521a    00000029                    : exit.obj (.text)
                  00095243    00000025                    : fs_toi28.obj (.text)
                  00095268    00000025                    : sinit.obj (.text)
                  0009528d    00000024                    : cpy_tbl.obj (.text)
                  000952b1    00000022                    : i_div28.obj (.text)
                  000952d3    00000020                    : new_.obj (.text)
                  000952f3    0000001d                    : memcpy.obj (.text)
                  00095310    0000001a                    : i_tofs28.obj (.text)
                  0009532a    00000019                    : args_main.obj (.text)
                  00095343    00000014                    : ll_mpy28.obj (.text)
                  00095357    0000000c                    : memset.obj (.text)
                  00095363    0000000b                    : u_div28.obj (.text)
                  0009536e    00000009                    : _lock.obj (.text)
                  00095377    00000008     F2807x_CodeStartBranch.obj (.text)
                  0009537f    00000005     rts2800_ml.lib : delete.obj (.text)
                  00095384    00000004                    : pure_virt.obj (.text)
                  00095388    00000003                    : error.obj (.text)
                  0009538b    00000002                    : pre_init.obj (.text)
                  0009538d    00000001                    : newhandler.obj (.text)
                  0009538e    00000001                    : startup.obj (.text)

ramfuncs   0    00095390    00000028     RUN ADDR = 0000b000
                  00095390    00000028     MainProcedure.obj (ramfuncs)

.econst    0    000953b8    00002091     
                  000953b8    000007d0     MainProcedure.obj (.econst:_iVbusInvTab)
                  00095b88    00000402     MainProcedure.obj (.econst:_InvSqrtTab)
                  00095f8a    00000402     MainProcedure.obj (.econst:_SqrtTab)
                  0009638c    0000034d     MainProcedure.obj (.econst:_PinMuxTable)
                  000966d9    00000001     --HOLE-- [fill = 0]
                  000966da    000001c0     MainProcedure.obj (.econst:_PieVectTableInit)
                  0009689a    00000169     MainProcedure.obj (.econst:_sintab)
                  00096a03    00000159     MainProcedure.obj (.econst:_VbpRangeTableForXfer208V)
                  00096b5c    00000159     MainProcedure.obj (.econst:_VbpRangeTableForXfer380V)
                  00096cb5    00000159     MainProcedure.obj (.econst:_VbpRangeTableForXfer400V)
                  00096e0e    000000e6     MainProcedure.obj (.econst:_Fbp50HzTableForXfer)
                  00096ef4    000000e6     MainProcedure.obj (.econst:_Fbp60HzTableForXfer)
                  00096fda    000000d1     MainProcedure.obj (.econst:_InvPointCntTab)
                  000970ab    000000cf     MainProcedure.obj (.econst:_VbpRangeTableForECOXfer)
                  0009717a    00000094     MainProcedure.obj (.econst:_CfgFromMonObjs1)
                  0009720e    00000068     MainProcedure.obj (.econst:_AlarmEventIdObj)
                  00097276    00000060     MainProcedure.obj (.econst:_CanCtrlMsgObjs)
                  000972d6    00000048     MainProcedure.obj (.econst:_CanAnlogMsgObjs)
                  0009731e    00000048     MainProcedure.obj (.econst:_CfgFromMonObjs2)
                  00097366    0000001e     MainProcedure.obj (.econst:_OtherInvNumTable)
                  00097384    00000017     MainProcedure.obj (.econst:_InvLoadTable)
                  0009739b    00000017     MainProcedure.obj (.econst:_OutLoadTable)
                  000973b2    00000014     MainProcedure.obj (.econst:_CanAnlogRecvMsgObjs)
                  000973c6    00000010     MainProcedure.obj (.econst:_CfgToMonObjs)
                  000973d6    00000010     MainProcedure.obj (.econst:_StateEventIdObj)
                  000973e6    00000010     MainProcedure.obj (.econst:_uInvSetMsgBitSet)
                  000973f6    0000000c     MainProcedure.obj (.econst:___vtbl__11CommandBase)
                  00097402    0000000c     MainProcedure.obj (.econst:___vtbl__14ProtocolSubCmd)
                  0009740e    0000000c     MainProcedure.obj (.econst:___vtbl__30TemplateCmd__tm__11_9SysCanApp)
                  0009741a    00000009     MainProcedure.obj (.econst:_g_ui16CANBitValues)
                  00097423    00000006     MainProcedure.obj (.econst)
                  00097429    00000001     --HOLE-- [fill = 0]
                  0009742a    00000004     MainProcedure.obj (.econst:_$P$T0)
                  0009742e    00000004     MainProcedure.obj (.econst:_$P$T1)
                  00097432    00000004     MainProcedure.obj (.econst:_$P$T2)
                  00097436    00000004     MainProcedure.obj (.econst:_$P$T3)
                  0009743a    00000004     MainProcedure.obj (.econst:_$P$T4)
                  0009743e    00000004     MainProcedure.obj (.econst:_Slicefor1stP)
                  00097442    00000004     MainProcedure.obj (.econst:_Slicefor1stQ)
                  00097446    00000003     MainProcedure.obj (.econst:_SliceforDC)

.CriticalIntFuncsSecured 
*          0    00097449    000005d9     RUN ADDR = 0000b050
                  00097449    000003f4     MainProcedure.obj (.CriticalIntFuncsSecured)
                  0009783d    000001e1     MainProcedure.obj (.CriticalIntFuncsSecured:retain)
                  00097a1e    00000004     F2807x_usDelay.obj (.CriticalIntFuncsSecured)

.cinit     0    00097a24    0000004d     
                  00097a24    0000001d     MainProcedure.obj (.cinit)
                  00097a41    0000000e     rts2800_ml.lib : exit.obj (.cinit)
                  00097a4f    00000008                    : atexit.obj (.cinit)
                  00097a57    00000005                    : _lock.obj (.cinit:__lock)
                  00097a5c    00000005                    : _lock.obj (.cinit:__unlock)
                  00097a61    00000005                    : sinit.obj (.cinit)
                  00097a66    00000005                    : vars.obj (.cinit)
                  00097a6b    00000004                    : memory.obj (.cinit)
                  00097a6f    00000002     --HOLE-- [fill = 0]

.switch    0    00097a74    00000046     
                  00097a74    00000028     MainProcedure.obj (.switch:_App_InvMaster__21Class_InverterControlFv)
                  00097a9c    0000001e     MainProcedure.obj (.switch:_App_MonInterfaceRead__22Class_MonitorInterfaceFv)

.pinit     0    00097abc    00000004     
                  00097abc    00000002     MainProcedure.obj (.pinit)
                  00097abe    00000002     --HOLE-- [fill = 0]

.stack     1    00000400    00000200     UNINITIALIZED
                  00000400    00000200     --HOLE--

AdcaResultFile 
*          1    00000b00    00000018     UNINITIALIZED
                  00000b00    00000018     MainProcedure.obj (AdcaResultFile)

AdcbResultFile 
*          1    00000b20    00000018     UNINITIALIZED
                  00000b20    00000018     MainProcedure.obj (AdcbResultFile)

AdcdResultFile 
*          1    00000b60    00000018     UNINITIALIZED
                  00000b60    00000018     MainProcedure.obj (AdcdResultFile)

CpuTimer0RegsFile 
*          1    00000c00    00000008     UNINITIALIZED
                  00000c00    00000008     MainProcedure.obj (CpuTimer0RegsFile)

CpuTimer1RegsFile 
*          1    00000c08    00000008     UNINITIALIZED
                  00000c08    00000008     MainProcedure.obj (CpuTimer1RegsFile)

CpuTimer2RegsFile 
*          1    00000c10    00000008     UNINITIALIZED
                  00000c10    00000008     MainProcedure.obj (CpuTimer2RegsFile)

PieCtrlRegsFile 
*          1    00000ce0    0000001a     UNINITIALIZED
                  00000ce0    0000001a     MainProcedure.obj (PieCtrlRegsFile)

PieVectTableFile 
*          1    00000d00    000001c0     UNINITIALIZED
                  00000d00    000001c0     MainProcedure.obj (PieVectTableFile)

EmuKeyVar 
*          1    00000d00    00000001     UNINITIALIZED
                  00000d00    00000001     MainProcedure.obj (EmuKeyVar)

EmuBModeVar 
*          1    00000d01    00000001     UNINITIALIZED
                  00000d01    00000001     MainProcedure.obj (EmuBModeVar)

FlashCallbackVar 
*          1    00000d02    00000000     UNINITIALIZED

FlashScalingVar 
*          1    00000d02    00000000     UNINITIALIZED

DmaRegsFile 
*          1    00001000    000000e0     UNINITIALIZED
                  00001000    000000e0     MainProcedure.obj (DmaRegsFile)

Cla1RegsFile 
*          1    00001400    0000003e     UNINITIALIZED
                  00001400    0000003e     MainProcedure.obj (Cla1RegsFile)

EPwm1RegsFile 
*          1    00004000    00000100     UNINITIALIZED
                  00004000    00000100     MainProcedure.obj (EPwm1RegsFile)

EPwm2RegsFile 
*          1    00004100    00000100     UNINITIALIZED
                  00004100    00000100     MainProcedure.obj (EPwm2RegsFile)

EPwm3RegsFile 
*          1    00004200    00000100     UNINITIALIZED
                  00004200    00000100     MainProcedure.obj (EPwm3RegsFile)

EPwm4RegsFile 
*          1    00004300    00000100     UNINITIALIZED
                  00004300    00000100     MainProcedure.obj (EPwm4RegsFile)

EPwm5RegsFile 
*          1    00004400    00000100     UNINITIALIZED
                  00004400    00000100     MainProcedure.obj (EPwm5RegsFile)

EPwm6RegsFile 
*          1    00004500    00000100     UNINITIALIZED
                  00004500    00000100     MainProcedure.obj (EPwm6RegsFile)

EPwm7RegsFile 
*          1    00004600    00000100     UNINITIALIZED
                  00004600    00000100     MainProcedure.obj (EPwm7RegsFile)

EPwm8RegsFile 
*          1    00004700    00000100     UNINITIALIZED
                  00004700    00000100     MainProcedure.obj (EPwm8RegsFile)

EPwm9RegsFile 
*          1    00004800    00000100     UNINITIALIZED
                  00004800    00000100     MainProcedure.obj (EPwm9RegsFile)

EPwm10RegsFile 
*          1    00004900    00000100     UNINITIALIZED
                  00004900    00000100     MainProcedure.obj (EPwm10RegsFile)

EPwm11RegsFile 
*          1    00004a00    00000100     UNINITIALIZED
                  00004a00    00000100     MainProcedure.obj (EPwm11RegsFile)

EPwm12RegsFile 
*          1    00004b00    00000100     UNINITIALIZED
                  00004b00    00000100     MainProcedure.obj (EPwm12RegsFile)

ECap1RegsFile 
*          1    00005000    00000020     UNINITIALIZED
                  00005000    00000020     MainProcedure.obj (ECap1RegsFile)

ECap2RegsFile 
*          1    00005020    00000020     UNINITIALIZED
                  00005020    00000020     MainProcedure.obj (ECap2RegsFile)

ECap3RegsFile 
*          1    00005040    00000020     UNINITIALIZED
                  00005040    00000020     MainProcedure.obj (ECap3RegsFile)

ECap4RegsFile 
*          1    00005060    00000020     UNINITIALIZED
                  00005060    00000020     MainProcedure.obj (ECap4RegsFile)

ECap5RegsFile 
*          1    00005080    00000020     UNINITIALIZED
                  00005080    00000020     MainProcedure.obj (ECap5RegsFile)

ECap6RegsFile 
*          1    000050a0    00000020     UNINITIALIZED
                  000050a0    00000020     MainProcedure.obj (ECap6RegsFile)

EQep1RegsFile 
*          1    00005100    00000022     UNINITIALIZED
                  00005100    00000022     MainProcedure.obj (EQep1RegsFile)

EQep2RegsFile 
*          1    00005140    00000022     UNINITIALIZED
                  00005140    00000022     MainProcedure.obj (EQep2RegsFile)

EQep3RegsFile 
*          1    00005180    00000022     UNINITIALIZED
                  00005180    00000022     MainProcedure.obj (EQep3RegsFile)

DacaRegsFile 
*          1    00005c00    00000008     UNINITIALIZED
                  00005c00    00000008     MainProcedure.obj (DacaRegsFile)

DacbRegsFile 
*          1    00005c10    00000008     UNINITIALIZED
                  00005c10    00000008     MainProcedure.obj (DacbRegsFile)

DaccRegsFile 
*          1    00005c20    00000008     UNINITIALIZED
                  00005c20    00000008     MainProcedure.obj (DaccRegsFile)

Cmpss1RegsFile 
*          1    00005c80    00000020     UNINITIALIZED
                  00005c80    00000020     MainProcedure.obj (Cmpss1RegsFile)

Cmpss2RegsFile 
*          1    00005ca0    00000020     UNINITIALIZED
                  00005ca0    00000020     MainProcedure.obj (Cmpss2RegsFile)

Cmpss3RegsFile 
*          1    00005cc0    00000020     UNINITIALIZED
                  00005cc0    00000020     MainProcedure.obj (Cmpss3RegsFile)

Cmpss4RegsFile 
*          1    00005ce0    00000020     UNINITIALIZED
                  00005ce0    00000020     MainProcedure.obj (Cmpss4RegsFile)

Cmpss5RegsFile 
*          1    00005d00    00000020     UNINITIALIZED
                  00005d00    00000020     MainProcedure.obj (Cmpss5RegsFile)

Cmpss6RegsFile 
*          1    00005d20    00000020     UNINITIALIZED
                  00005d20    00000020     MainProcedure.obj (Cmpss6RegsFile)

Cmpss7RegsFile 
*          1    00005d40    00000020     UNINITIALIZED
                  00005d40    00000020     MainProcedure.obj (Cmpss7RegsFile)

Cmpss8RegsFile 
*          1    00005d60    00000020     UNINITIALIZED
                  00005d60    00000020     MainProcedure.obj (Cmpss8RegsFile)

Sdfm1RegsFile 
*          1    00005e00    00000080     UNINITIALIZED
                  00005e00    00000080     MainProcedure.obj (Sdfm1RegsFile)

Sdfm2RegsFile 
*          1    00005e80    00000080     UNINITIALIZED
                  00005e80    00000080     MainProcedure.obj (Sdfm2RegsFile)

McbspaRegsFile 
*          1    00006000    00000024     UNINITIALIZED
                  00006000    00000024     MainProcedure.obj (McbspaRegsFile)

McbspbRegsFile 
*          1    00006040    00000024     UNINITIALIZED
                  00006040    00000024     MainProcedure.obj (McbspbRegsFile)

SpiaRegsFile 
*          1    00006100    00000010     UNINITIALIZED
                  00006100    00000010     MainProcedure.obj (SpiaRegsFile)

SpibRegsFile 
*          1    00006110    00000010     UNINITIALIZED
                  00006110    00000010     MainProcedure.obj (SpibRegsFile)

SpicRegsFile 
*          1    00006120    00000010     UNINITIALIZED
                  00006120    00000010     MainProcedure.obj (SpicRegsFile)

WdRegsFile 
*          1    00007000    0000002b     UNINITIALIZED
                  00007000    0000002b     MainProcedure.obj (WdRegsFile)

NmiIntruptRegsFile 
*          1    00007060    00000007     UNINITIALIZED
                  00007060    00000007     MainProcedure.obj (NmiIntruptRegsFile)

XintRegsFile 
*          1    00007070    0000000b     UNINITIALIZED
                  00007070    0000000b     MainProcedure.obj (XintRegsFile)

SciaRegsFile 
*          1    00007200    00000010     UNINITIALIZED
                  00007200    00000010     MainProcedure.obj (SciaRegsFile)

ScibRegsFile 
*          1    00007210    00000010     UNINITIALIZED
                  00007210    00000010     MainProcedure.obj (ScibRegsFile)

ScicRegsFile 
*          1    00007220    00000010     UNINITIALIZED
                  00007220    00000010     MainProcedure.obj (ScicRegsFile)

ScidRegsFile 
*          1    00007230    00000010     UNINITIALIZED
                  00007230    00000010     MainProcedure.obj (ScidRegsFile)

I2caRegsFile 
*          1    00007300    00000022     UNINITIALIZED
                  00007300    00000022     MainProcedure.obj (I2caRegsFile)

I2cbRegsFile 
*          1    00007340    00000022     UNINITIALIZED
                  00007340    00000022     MainProcedure.obj (I2cbRegsFile)

AdcaRegsFile 
*          1    00007400    00000080     UNINITIALIZED
                  00007400    00000080     MainProcedure.obj (AdcaRegsFile)

AdcbRegsFile 
*          1    00007480    00000080     UNINITIALIZED
                  00007480    00000080     MainProcedure.obj (AdcbRegsFile)

AdcdRegsFile 
*          1    00007580    00000080     UNINITIALIZED
                  00007580    00000080     MainProcedure.obj (AdcdRegsFile)

InputXbarRegsFile 
*          1    00007900    00000020     UNINITIALIZED
                  00007900    00000020     MainProcedure.obj (InputXbarRegsFile)

XbarRegsFile 
*          1    00007920    00000020     UNINITIALIZED
                  00007920    00000020     MainProcedure.obj (XbarRegsFile)

SyncSocRegsFile 
*          1    00007940    00000006     UNINITIALIZED
                  00007940    00000006     MainProcedure.obj (SyncSocRegsFile)

DmaClaSrcSelRegsFile 
*          1    00007980    0000001a     UNINITIALIZED
                  00007980    0000001a     MainProcedure.obj (DmaClaSrcSelRegsFile)

EPwmXbarRegsFile 
*          1    00007a00    00000040     UNINITIALIZED
                  00007a00    00000040     MainProcedure.obj (EPwmXbarRegsFile)

OutputXbarRegsFile 
*          1    00007a80    00000040     UNINITIALIZED
                  00007a80    00000040     MainProcedure.obj (OutputXbarRegsFile)

GpioCtrlRegsFile 
*          1    00007c00    00000180     UNINITIALIZED
                  00007c00    00000180     MainProcedure.obj (GpioCtrlRegsFile)

GpioDataRegsFile 
*          1    00007f00    00000030     UNINITIALIZED
                  00007f00    00000030     MainProcedure.obj (GpioDataRegsFile)

.ebss      1    0000c000    00001ac4     UNINITIALIZED
                  0000c000    000019ae     MainProcedure.obj (.ebss)
                  0000d9ae    00000008     rts2800_ml.lib : memory.obj (.ebss)
                  0000d9b6    00000006                    : exit.obj (.ebss)
                  0000d9bc    00000002                    : _lock.obj (.ebss:__lock)
                  0000d9be    00000002                    : _lock.obj (.ebss:__unlock)
                  0000d9c0    00000100                    : atexit.obj (.ebss)
                  0000dac0    00000002                    : sinit.obj (.ebss)
                  0000dac2    00000002                    : vars.obj (.ebss)

.esysmem   1    0000e800    00000400     UNINITIALIZED
                  0000e800    00000001     rts2800_ml.lib : memory.obj (.esysmem)
                  0000e801    000003ff     --HOLE--

.reset     0    003fffc0    00000002     DSECT
                  003fffc0    00000002     rts2800_ml.lib : boot28.obj (.reset)

.FaultRecord 
*          1    00012000    00000180     UNINITIALIZED
                  00012000    00000180     MainProcedure.obj (.FaultRecord)

.DSPflashdata 
*          1    00012000    00000c60     UNINITIALIZED
                  00012000    00000c60     MainProcedure.obj (.DSPflashdata)

.FPGAflashdata 
*          1    00012000    00000082     UNINITIALIZED
                  00012000    00000082     MainProcedure.obj (.FPGAflashdata)

.FPGAEEPROMdata 
*          1    00012f00    00000082     UNINITIALIZED
                  00012f00    00000082     MainProcedure.obj (.FPGAEEPROMdata)

AnalogSubsysRegsFile 
*          1    0005d180    00000048     UNINITIALIZED
                  0005d180    00000048     MainProcedure.obj (AnalogSubsysRegsFile)

Cla1SoftIntRegsFile 
*          1    00000ce0    00000004     DSECT
                  00000ce0    00000004     MainProcedure.obj (Cla1SoftIntRegsFile)

Emif1RegsFile 
*          1    00047000    00000070     UNINITIALIZED
                  00047000    00000070     MainProcedure.obj (Emif1RegsFile)

DevCfgRegsFile 
*          1    0005d000    0000012e     UNINITIALIZED
                  0005d000    0000012e     MainProcedure.obj (DevCfgRegsFile)

ClkCfgRegsFile 
*          1    0005d200    00000032     UNINITIALIZED
                  0005d200    00000032     MainProcedure.obj (ClkCfgRegsFile)

CpuSysRegsFile 
*          1    0005d300    00000082     UNINITIALIZED
                  0005d300    00000082     MainProcedure.obj (CpuSysRegsFile)

RomPrefetchRegsFile 
*          1    0005e608    00000002     UNINITIALIZED
                  0005e608    00000002     MainProcedure.obj (RomPrefetchRegsFile)

DcsmZ1RegsFile 
*          1    0005f000    00000024     UNINITIALIZED
                  0005f000    00000024     MainProcedure.obj (DcsmZ1RegsFile)

DcsmZ2RegsFile 
*          1    0005f040    00000024     UNINITIALIZED
                  0005f040    00000024     MainProcedure.obj (DcsmZ2RegsFile)

DcsmCommonRegsFile 
*          1    0005f070    00000008     UNINITIALIZED
                  0005f070    00000008     MainProcedure.obj (DcsmCommonRegsFile)

MemCfgRegsFile 
*          1    0005f400    00000080     UNINITIALIZED
                  0005f400    00000080     MainProcedure.obj (MemCfgRegsFile)

Emif1ConfigRegsFile 
*          1    0005f480    00000020     UNINITIALIZED
                  0005f480    00000020     MainProcedure.obj (Emif1ConfigRegsFile)

AccessProtectionRegsFile 
*          1    0005f4c0    00000040     UNINITIALIZED
                  0005f4c0    00000040     MainProcedure.obj (AccessProtectionRegsFile)

MemoryErrorRegsFile 
*          1    0005f500    00000040     UNINITIALIZED
                  0005f500    00000040     MainProcedure.obj (MemoryErrorRegsFile)

RomWaitStateRegsFile 
*          1    0005f540    00000002     UNINITIALIZED
                  0005f540    00000002     MainProcedure.obj (RomWaitStateRegsFile)

Flash0CtrlRegsFile 
*          1    0005f800    00000182     UNINITIALIZED
                  0005f800    00000182     MainProcedure.obj (Flash0CtrlRegsFile)

Flash0EccRegsFile 
*          1    0005fb00    00000028     UNINITIALIZED
                  0005fb00    00000028     MainProcedure.obj (Flash0EccRegsFile)

DcsmZ1OtpFile 
*          1    00078000    00000020     NOLOAD SECTION
                  00078000    00000020     MainProcedure.obj (DcsmZ1OtpFile)

DcsmZ2OtpFile 
*          1    00078200    00000020     NOLOAD SECTION
                  00078200    00000020     MainProcedure.obj (DcsmZ2OtpFile)

MODULE SUMMARY

       Module                       code    initialized data   uninitialized data
       ------                       ----    ----------------   ------------------
    .\
       MainProcedure.obj            84395   8948               18027             
       F2807x_CodeStartBranch.obj   10      0                  0                 
       F2807x_usDelay.obj           8       0                  0                 
    +--+----------------------------+-------+------------------+--------------------+
       Total:                       84413   8948               18027             
                                                                                 
    E:\ti\ccsv7\tools\compiler\ti-cgt-c2000_16.9.1.LTS\lib\rts2800_ml.lib
       memory.obj                   461     4                  8                 
       atexit.obj                   0       8                  256               
       ll_div28.obj                 263     0                  0                 
       fs_div28.obj                 131     0                  0                 
       fs_mpy28.obj                 90      0                  0                 
       boot28.obj                   84      0                  0                 
       exit.obj                     41      14                 6                 
       sinit.obj                    37      5                  2                 
       l_div28.obj                  42      0                  0                 
       fs_toi28.obj                 37      0                  0                 
       cpy_tbl.obj                  36      0                  0                 
       i_div28.obj                  34      0                  0                 
       new_.obj                     32      0                  0                 
       memcpy.obj                   29      0                  0                 
       i_tofs28.obj                 26      0                  0                 
       args_main.obj                25      0                  0                 
       _lock.obj                    9       10                 4                 
       ll_mpy28.obj                 20      0                  0                 
       memset.obj                   12      0                  0                 
       u_div28.obj                  11      0                  0                 
       vars.obj                     0       5                  2                 
       delete.obj                   5       0                  0                 
       pure_virt.obj                4       0                  0                 
       error.obj                    3       0                  0                 
       pre_init.obj                 2       0                  0                 
       newhandler.obj               1       0                  0                 
       startup.obj                  1       0                  0                 
    +--+----------------------------+-------+------------------+--------------------+
       Total:                       1436    46                 278               
                                                                                 
       Heap:                        0       0                  1024              
       Stack:                       0       0                  512               
    +--+----------------------------+-------+------------------+--------------------+
       Grand Total:                 85849   8994               19841             


GLOBAL DATA SYMBOLS: SORTED BY DATA PAGE

address     data page           name
--------    ----------------    ----
00000400      10 (00000400)     __stack

00000b00      2c (00000b00)     _AdcaResultRegs
00000b20      2c (00000b00)     _AdcbResultRegs

00000b60      2d (00000b40)     _AdcdResultRegs

00000c00      30 (00000c00)     _CpuTimer0Regs
00000c08      30 (00000c00)     _CpuTimer1Regs
00000c10      30 (00000c00)     _CpuTimer2Regs

00000ce0      33 (00000cc0)     _Cla1SoftIntRegs
00000ce0      33 (00000cc0)     _PieCtrlRegs

00000d00      34 (00000d00)     _EmuKey
00000d00      34 (00000d00)     _PieVectTable
00000d01      34 (00000d00)     _EmuBMode

00001000      40 (00001000)     _DmaRegs

00001400      50 (00001400)     _Cla1Regs

00004000     100 (00004000)     _EPwm1Regs

00004100     104 (00004100)     _EPwm2Regs

00004200     108 (00004200)     _EPwm3Regs

00004300     10c (00004300)     _EPwm4Regs

00004400     110 (00004400)     _EPwm5Regs

00004500     114 (00004500)     _EPwm6Regs

00004600     118 (00004600)     _EPwm7Regs

00004700     11c (00004700)     _EPwm8Regs

00004800     120 (00004800)     _EPwm9Regs

00004900     124 (00004900)     _EPwm10Regs

00004a00     128 (00004a00)     _EPwm11Regs

00004b00     12c (00004b00)     _EPwm12Regs

00005000     140 (00005000)     _ECap1Regs
00005020     140 (00005000)     _ECap2Regs

00005040     141 (00005040)     _ECap3Regs
00005060     141 (00005040)     _ECap4Regs

00005080     142 (00005080)     _ECap5Regs
000050a0     142 (00005080)     _ECap6Regs

00005100     144 (00005100)     _EQep1Regs

00005140     145 (00005140)     _EQep2Regs

00005180     146 (00005180)     _EQep3Regs

00005c00     170 (00005c00)     _DacaRegs
00005c10     170 (00005c00)     _DacbRegs
00005c20     170 (00005c00)     _DaccRegs

00005c80     172 (00005c80)     _Cmpss1Regs
00005ca0     172 (00005c80)     _Cmpss2Regs

00005cc0     173 (00005cc0)     _Cmpss3Regs
00005ce0     173 (00005cc0)     _Cmpss4Regs

00005d00     174 (00005d00)     _Cmpss5Regs
00005d20     174 (00005d00)     _Cmpss6Regs

00005d40     175 (00005d40)     _Cmpss7Regs
00005d60     175 (00005d40)     _Cmpss8Regs

00005e00     178 (00005e00)     _Sdfm1Regs

00005e80     17a (00005e80)     _Sdfm2Regs

00006000     180 (00006000)     _McbspaRegs

00006040     181 (00006040)     _McbspbRegs

00006100     184 (00006100)     _SpiaRegs
00006110     184 (00006100)     _SpibRegs
00006120     184 (00006100)     _SpicRegs

00007000     1c0 (00007000)     _WdRegs

00007060     1c1 (00007040)     _NmiIntruptRegs
00007070     1c1 (00007040)     _XintRegs

00007200     1c8 (00007200)     _SciaRegs
00007210     1c8 (00007200)     _ScibRegs
00007220     1c8 (00007200)     _ScicRegs
00007230     1c8 (00007200)     _ScidRegs

00007300     1cc (00007300)     _I2caRegs

00007340     1cd (00007340)     _I2cbRegs

00007400     1d0 (00007400)     _AdcaRegs

00007480     1d2 (00007480)     _AdcbRegs

00007580     1d6 (00007580)     _AdcdRegs

00007900     1e4 (00007900)     _InputXbarRegs
00007920     1e4 (00007900)     _XbarRegs

00007940     1e5 (00007940)     _SyncSocRegs

00007980     1e6 (00007980)     _DmaClaSrcSelRegs

00007a00     1e8 (00007a00)     _EPwmXbarRegs

00007a80     1ea (00007a80)     _OutputXbarRegs

00007c00     1f0 (00007c00)     _GpioCtrlRegs

00007f00     1fc (00007f00)     _GpioDataRegs

0000c000     300 (0000c000)     _objRAMDrv
0000c001     300 (0000c000)     _objPWMDrv
0000c002     300 (0000c000)     _objSCIDrv
0000c003     300 (0000c000)     _objCMPSSDrv
0000c004     300 (0000c000)     _objWatchDogDrv
0000c005     300 (0000c000)     _objCLA
0000c006     300 (0000c000)     _objCANDrv
0000c007     300 (0000c000)     _objI2CDrv
0000c008     300 (0000c000)     _objFlashDrv
0000c009     300 (0000c000)     _objCAPDrv
0000c00a     300 (0000c000)     _objGPIODrv
0000c00b     300 (0000c000)     _g_u16_INTRunTime
0000c00c     300 (0000c000)     _g_u16_MainRunTimeMax
0000c00d     300 (0000c000)     _g_u16_INTRunTimeMax
0000c00e     300 (0000c000)     _g_i16_IntCnt1Per4_0
0000c00f     300 (0000c000)     _g_i16_IntCnt1Per2_0
0000c010     300 (0000c000)     _objPowCANPro
0000c011     300 (0000c000)     _objFlashUpdate
0000c012     300 (0000c000)     _objECO
0000c013     300 (0000c000)     _g_u16_MainRunTime
0000c014     300 (0000c000)     _u16_FPGA_Flash_CANInit
0000c015     300 (0000c000)     _objService
0000c017     300 (0000c000)     _objSysDrv
0000c01a     300 (0000c000)     _pCanIsrXmitFcb
0000c01c     300 (0000c000)     _m_pDataExchgPtr__15SysCanDataExchg
0000c01e     300 (0000c000)     _pCanIsrRecvFcb
0000c020     300 (0000c000)     _g_ulRxMsgCount
0000c022     300 (0000c000)     _g_bErrFlag
0000c024     300 (0000c000)     _g_ulTxMsgCount
0000c026     300 (0000c000)     _objFaultRecord
0000c02a     300 (0000c000)     _objFPGAConfig
0000c034     300 (0000c000)     _ReceiveFrame

0000c040     301 (0000c040)     _objParallel
0000c047     301 (0000c040)     _ucRXAMsgData
0000c04f     301 (0000c040)     _ucTXAMsgData
0000c057     301 (0000c040)     _ucRXBMsgData
0000c05f     301 (0000c040)     _ucTXBMsgData
0000c067     301 (0000c040)     _objTimerDrv
0000c070     301 (0000c040)     _sTXCANAMessage

0000c080     302 (0000c080)     _sRXCANBMessage
0000c08a     302 (0000c080)     _sRXCANAMessage
0000c094     302 (0000c080)     _sTXCANBMessage
0000c09e     302 (0000c080)     _objLBS
0000c0ac     302 (0000c080)     _objDCBus

0000c0c0     303 (0000c0c0)     _objSwitches
0000c0cf     303 (0000c0c0)     _objInvCtrl
0000c0de     303 (0000c0c0)     _uInvAnalogLen

0000c100     304 (0000c100)     _objSPIDrv

0000c140     305 (0000c140)     _objXfer

0000c180     306 (0000c180)     _objEEPROM

0000c1c0     307 (0000c1c0)     _objADCDrv

0000c200     308 (0000c200)     _objLoad

0000c240     309 (0000c240)     _objSelfAgingAlg

0000c280     30a (0000c280)     _objDebug

0000c2c0     30b (0000c2c0)     _objDigitalIO

0000c340     30d (0000c340)     _objBypass

0000c3c0     30f (0000c3c0)     _objOutput

0000c480     312 (0000c480)     _objInvAlg

0000c540     315 (0000c540)     _objSystem

0000c600     318 (0000c600)     _objMonInterface

0000c700     31c (0000c700)     _objSysCanApp

0000c840     321 (0000c840)     _objFPGAFlash

0000ca40     329 (0000ca40)     _objPowCANSched

0000cc80     332 (0000cc80)     _objProtocol

0000cf80     33e (0000cf80)     _objDataExchg

0000d340     34d (0000d340)     _objInverter

0000d9b6     366 (0000d980)     ___TI_enable_exit_profile_output
0000d9b8     366 (0000d980)     ___TI_cleanup_ptr
0000d9ba     366 (0000d980)     ___TI_dtors_ptr
0000d9bc     366 (0000d980)     __lock
0000d9be     366 (0000d980)     __unlock

0000d9c1     367 (0000d9c0)     ___atexit_func_id__

0000dac2     36b (0000dac0)     __new_handler

0000e800     3a0 (0000e800)     __sys_memory

00012000     480 (00012000)     _DebugRxBuff
00012000     480 (00012000)     _FPGACodeEEPROMBuff
00012000     480 (00012000)     _uFaultRecord

00012080     482 (00012080)     _u16FaultRecordRead

000120c0     483 (000120c0)     _byCRCLoArrayFlash

00012100     484 (00012100)     _uFaultRecordBuff

000121c0     487 (000121c0)     _byCRCHiArrayFlash

000122c0     48b (000122c0)     _m_u16_SCIRxBuff

00012400     490 (00012400)     _FlashBuffer

00012800     4a0 (00012800)     _st_FlashVariable

00012f00     4bc (00012f00)     _DebugEEPROMBuff

00047000    11c0 (00047000)     _Emif1Regs

0005d000    1740 (0005d000)     _DevCfgRegs

0005d180    1746 (0005d180)     _AnalogSubsysRegs

0005d200    1748 (0005d200)     _ClkCfgRegs

0005d300    174c (0005d300)     _CpuSysRegs

0005e608    1798 (0005e600)     _RomPrefetchRegs

0005f000    17c0 (0005f000)     _DcsmZ1Regs

0005f040    17c1 (0005f040)     _DcsmZ2Regs
0005f070    17c1 (0005f040)     _DcsmCommonRegs

0005f400    17d0 (0005f400)     _MemCfgRegs

0005f480    17d2 (0005f480)     _Emif1ConfigRegs

0005f4c0    17d3 (0005f4c0)     _AccessProtectionRegs

0005f500    17d4 (0005f500)     _MemoryErrorRegs

0005f540    17d5 (0005f540)     _RomWaitStateRegs

0005f800    17e0 (0005f800)     _Flash0CtrlRegs

0005fb00    17ec (0005fb00)     _Flash0EccRegs

00078000    1e00 (00078000)     _DcsmZ1Otp

00078200    1e08 (00078200)     _DcsmZ2Otp

00097402    25d0 (00097400)     ___vtbl__14ProtocolSubCmd
0009740e    25d0 (00097400)     ___vtbl__30TemplateCmd__tm__11_9SysCanApp


GLOBAL SYMBOLS: SORTED ALPHABETICALLY BY Name 

page  address   name                                                                                   
----  -------   ----                                                                                   
0     00086b40  .text                                                                                  
0     0009521a  C$$EXIT                                                                                
abs   00000100  CLA_SCRATCHPAD_SIZE                                                                    
0     000950bf  FS$$DIV                                                                                
0     00095142  FS$$MPY                                                                                
0     00095243  FS$$TOI                                                                                
0     000952b1  I$$DIV                                                                                 
0     000952c2  I$$MOD                                                                                 
0     00095310  I$$TOFS                                                                                
0     000951f0  L$$DIV                                                                                 
0     000951ff  L$$MOD                                                                                 
0     00094fb8  LL$$DIV                                                                                
0     00094ff4  LL$$MOD                                                                                
0     00095343  LL$$MPY                                                                                
0     00095363  U$$DIV                                                                                 
0     00095368  U$$MOD                                                                                 
0     0009520d  UL$$DIV                                                                                
0     00095214  UL$$MOD                                                                                
0     0009502e  ULL$$DIV                                                                               
0     0009505d  ULL$$MOD                                                                               
0     00094ab4  _ADCA1_ISR                                                                             
0     00094bef  _ADCA2_ISR                                                                             
0     00094bf4  _ADCA3_ISR                                                                             
0     00094bf9  _ADCA4_ISR                                                                             
0     00094bea  _ADCA_EVT_ISR                                                                          
0     00094ab9  _ADCB1_ISR                                                                             
0     00094c03  _ADCB2_ISR                                                                             
0     00094c08  _ADCB3_ISR                                                                             
0     00094c0d  _ADCB4_ISR                                                                             
0     00094bfe  _ADCB_EVT_ISR                                                                          
0     00094ac8  _ADCD1_ISR                                                                             
0     00094cb2  _ADCD2_ISR                                                                             
0     00094cb7  _ADCD3_ISR                                                                             
0     00094cbc  _ADCD4_ISR                                                                             
0     00094cad  _ADCD_EVT_ISR                                                                          
0     00089fe0  _APP_EcoInvBpStatusF__12Class_SystemFv                                                 
0     00089d7f  _APP_ModulePWMMicroAdj__12Class_SystemFv                                               
0     00094cda  _AUX_PLL_SLIP_ISR                                                                      
0     0009399e  _AbnormalShutCancelCmd__15SysCanDataExchgFv                                            
0     0009398c  _AbnormalShutConfirmCmd__15SysCanDataExchgFv                                           
1     0005f4c0  _AccessProtectionRegs                                                                  
1     00007400  _AdcaRegs                                                                              
1     00000b00  _AdcaResultRegs                                                                        
1     00007480  _AdcbRegs                                                                              
1     00000b20  _AdcbResultRegs                                                                        
1     00007580  _AdcdRegs                                                                              
1     00000b60  _AdcdResultRegs                                                                        
0     00092f9b  _AlarmEventXmitMsgGen__15SysCanDataExchgFUi                                            
0     0008becb  _Alg_BpFault__12Class_BypassFv                                                         
0     0008be70  _Alg_BpSeqFault__12Class_BypassFv                                                      
0     0008d06f  _Alg_DCBusFault__11Class_DCBusFv                                                       
0     00089d00  _Alg_HeatFault__12Class_SystemFv                                                       
0     0008ad32  _Alg_INVKMFastChk__14Class_SwitchesFv                                                  
0     00090c53  _Alg_Int_AgingSPWM__24Class_SelfAgingAlgorithmFv                                       
0     0000f176  _Alg_Int_CarrierPowerCANSync__23Class_InverterAlgorithmFv                              
0     000114ed  _Alg_Int_DCOVProtect__11Class_DCBusFv                                                  
0     0000fc22  _Alg_Int_ECOFreqFastChk__23Class_InverterAlgorithmFv                                   
0     0000f102  _Alg_Int_InvOffReset__23Class_InverterAlgorithmFv                                      
0     0000f8b0  _Alg_Int_InvSyncPulseGen__23Class_InverterAlgorithmFv                                  
0     0000f9c1  _Alg_Int_InvSyncPulseRec__23Class_InverterAlgorithmFv                                  
0     0000fa86  _Alg_Int_InvSyncRecord__23Class_InverterAlgorithmFv                                    
0     00011765  _Alg_Int_LBSDetect__9Class_LBSFv                                                       
0     0000fa98  _Alg_Int_LockStatus__23Class_InverterAlgorithmFv                                       
0     0000f285  _Alg_Int_PhaseLock1__23Class_InverterAlgorithmFv                                       
0     0001059d  _Alg_Int_STSDiffFastChk__14Class_SwitchesFv                                            
0     00090c30  _Alg_Int_SelfAging__24Class_SelfAgingAlgorithmFv                                       
0     00011327  _Alg_Int_VoutAbnormal__12Class_OutputFv                                                
0     00010f3a  _Alg_Int_VoutFastChk__12Class_OutputFv                                                 
0     0008c97f  _Alg_InvFault__14Class_InverterFv                                                      
0     0008c9e7  _Alg_InvOverCurrentChk__14Class_InverterFv                                             
0     00090252  _Alg_LBSSignal__9Class_LBSFv                                                           
0     00089965  _Alg_OperFault__12Class_SystemFv                                                       
0     0008cfd1  _Alg_ParaFault__14Class_ParallelFv                                                     
0     0008cf37  _Alg_ParaStatus__14Class_ParallelFv                                                    
0     0008b09b  _Alg_STSOpenFault__14Class_SwitchesFv                                                  
0     0008ae39  _Alg_STSShortFault__14Class_SwitchesFv                                                 
0     0008e7af  _Alg_ShortCircuitDetect__10Class_LoadFv                                                
0     000898bf  _Alg_SysFault__12Class_SystemFv                                                        
0     0008ceaa  _Alg_VoutAbnormal__12Class_OutputFv                                                    
0     0008ca7d  _Alg_VoutToGnd_Fault__14Class_InverterFv                                               
0     00092e2c  _AlrmCovMsgXmitState__15SysCanDataExchgFi                                              
0     000936a1  _AlrmMsgRecvProc__15SysCanDataExchgFP19can_msg_data_struct                             
0     000932ac  _AlrmSyncMsgXmitState__15SysCanDataExchgFi                                             
0     00092e3b  _AlrmXmitMsgGen__15SysCanDataExchgFUi                                                  
0     00093aed  _AnalogMsgRecvProc__15SysCanDataExchgFP19can_msg_data_struct                           
0     00093b6a  _AnalogRecvMsgObjsInit__15SysCanDataExchgFv                                            
1     0005d180  _AnalogSubsysRegs                                                                      
0     00093311  _AnalogSyncMsgXmitState__15SysCanDataExchgFi                                           
0     00093d73  _AnalogXmitMsgGen__15SysCanDataExchgFUi                                                
0     00091fc3  _AppSubCmdIni__9AppSubCmdFP9SysCanAppM9SysCanAppFPv_i                                  
0     0008b203  _App_BpParamConfig__12Class_BypassFv                                                   
0     0008b19a  _App_BpVarInit__12Class_BypassFv                                                       
0     0008d00e  _App_DCBusParamConfig__11Class_DCBusFv                                                 
0     0008cff7  _App_DCBusVarInit__11Class_DCBusFv                                                     
0     0008971c  _App_DSPCheck__12Class_SystemFv                                                        
0     00090a04  _App_DSPResetInfoWrite__12Class_EEPROMFv                                               
0     0000b263  _App_DSPRestart__17Class_FlashUpdateFv                                                 
0     00090da3  _App_DebugVarInit__11Class_DebugFv                                                     
0     0000b0a1  _App_Delay1ms__17Class_FlashUpdateFv                                                   
0     0000b0ba  _App_Delay20ms__17Class_FlashUpdateFv                                                  
0     0008a451  _App_DigitalIOVarInit__15Class_DigitalIOFv                                             
0     00090343  _App_ECOInvToBpFlagDeal__9Class_ECOFv                                                  
0     0009033d  _App_ECO__9Class_ECOFv                                                                 
0     00090a9d  _App_EEPROMAction__12Class_EEPROMFv                                                    
0     00090984  _App_EEPROMRead__12Class_EEPROMFv                                                      
0     00090ae4  _App_EEPROMVerify__12Class_EEPROMFPUiT1Ui                                              
0     000909b9  _App_EEPROMWrite__12Class_EEPROMFv                                                     
0     000910d3  _App_FPGAConfigError__16Class_FPGAConfigFUi                                            
0     00090f99  _App_FPGAConfigProcess__16Class_FPGAConfigFv                                           
0     00091ca6  _App_FPGAFlashMain_CAN__15Class_FPGAFlashFv                                            
0     00089753  _App_FPGA_Ver__12Class_SystemFv                                                        
0     00089c90  _App_FanNeedHighSpeed__12Class_SystemFv                                                
0     00090853  _App_FaultEEPROMW__12Class_EEPROMFv                                                    
0     00090905  _App_FaultReadTaskInit__12Class_EEPROMFi                                               
0     000908e3  _App_FaultRead__12Class_EEPROMFv                                                       
0     000903af  _App_FaultRecordTaxsis__17Class_FaultRecordFv                                          
0     00090481  _App_FaultRecord__17Class_FaultRecordFv                                                
0     0000b081  _App_FlashAPIInit__17Class_FlashUpdateFv                                               
0     0000b08f  _App_FlashUpdateMain__17Class_FlashUpdateFv                                            
0     0000b093  _App_Flash_CsmUnlock__17Class_FlashUpdateFv                                            
0     00089fb4  _App_FwupdateCondition__12Class_SystemFv                                               
0     0008aa63  _App_IMCCtrl__15Class_DigitalIOFv                                                      
0     00010262  _App_Int_Can_SendSchedule__21Class_PowCANSchedulerFv                                   
0     0000fcb1  _App_Int_CurrSharOptPreDeal_Route1__21Class_PowCANSchedulerFv                          
0     000115ee  _App_Int_ECOInvSoftstart__21Class_InverterControlFv                                    
0     0001167d  _App_Int_FlagCntReset__21Class_InverterControlFv                                       
0     00010d21  _App_Int_InvOffReset__14Class_InverterFv                                               
0     00010542  _App_Int_SPIAct__15Class_DigitalIOFv                                                   
0     00011a62  _App_Int_SciFrameReceive__15Class_FPGAFlashFv                                          
0     000119a9  _App_Int_VirtualScopeStartup__11Class_DebugFv                                          
0     0001178f  _App_Int_WaveRecord__11Class_DebugFv                                                   
0     000899a9  _App_IntelligentParall__12Class_SystemFv                                               
0     0008881c  _App_InvAlgParamConfig1__23Class_InverterAlgorithmFv                                   
0     00088b9d  _App_InvAlgParamConfig2__23Class_InverterAlgorithmFv                                   
0     0008879b  _App_InvAlgVarInit__23Class_InverterAlgorithmFv                                        
0     0008ee10  _App_InvCtrl__21Class_InverterControlFv                                                
0     0008f13e  _App_InvMaster__21Class_InverterControlFv                                              
0     0008ee30  _App_InvOffReason__21Class_InverterControlFv                                           
0     0008f030  _App_InvOnoffAction__21Class_InverterControlFv                                         
0     0008ee81  _App_InvOnoffAgent__21Class_InverterControlFv                                          
0     0008c052  _App_InvParamConfig__14Class_InverterFv                                                
0     0008f28d  _App_InvSoftstart__21Class_InverterControlFv                                           
0     0008f360  _App_InvStandby__21Class_InverterControlFv                                             
0     0008f276  _App_InvTrace__21Class_InverterControlFv                                               
0     0008bfc6  _App_InvVarInit__14Class_InverterFv                                                    
0     00089d59  _App_LimitPulseByPulseSet__12Class_SystemFv                                            
0     0008952d  _App_ModuleOnline__12Class_SystemFv                                                    
0     00089a10  _App_ModuleRelax_Affirm__12Class_SystemFv                                              
0     000897dc  _App_Module_LED__12Class_SystemFv                                                      
0     00089776  _App_Module_Ok__12Class_SystemFv                                                       
0     0008df9a  _App_MonInterfaceRead__22Class_MonitorInterfaceFv                                      
0     0008d5ab  _App_MonInterfaceWrite__22Class_MonitorInterfaceFv                                     
0     0008d58b  _App_MonitorDeal__22Class_MonitorInterfaceFv                                           
0     0008db82  _App_MonitorOrder__22Class_MonitorInterfaceFv                                          
0     0008df26  _App_MonitorParam__22Class_MonitorInterfaceFv                                          
0     0008d15a  _App_MonitorVarInit__22Class_MonitorInterfaceFv                                        
0     0008cb16  _App_OutParamConfig__12Class_OutputFv                                                  
0     0008cac9  _App_OutVarInit__12Class_OutputFv                                                      
0     0008ec83  _App_OvloadDelay__10Class_LoadFv                                                       
0     0008edcd  _App_OvloadSignal__10Class_LoadFv                                                      
0     0008e6a7  _App_ParallelLocalData__22Class_MonitorInterfaceFv                                     
0     0009069c  _App_ParamEEPROMW__12Class_EEPROMFv                                                    
0     00090953  _App_ParamReadTaskInit__12Class_EEPROMFv                                               
0     0008a3ea  _App_PowCANConfigUpdate__21Class_PowCANSchedulerFv                                     
0     0008a028  _App_PowCANInit__21Class_PowCANSchedulerFv                                             
0     00089b00  _App_Relax_Command__12Class_SystemFv                                                   
0     00091b5b  _App_SCIVarInit__15Class_FPGAFlashFv                                                   
0     000910e5  _App_SciFlashMain__15Class_FPGAFlashFv                                                 
0     00090b24  _App_SelfAgingAlgParamConfig__24Class_SelfAgingAlgorithmFv                             
0     00090b07  _App_SelfAgingAlgVarInit__24Class_SelfAgingAlgorithmFv                                 
0     00090be9  _App_SelfAgingTargetUpdate__24Class_SelfAgingAlgorithmFv                               
0     0008ddd2  _App_SendtoMonitor__22Class_MonitorInterfaceFv                                         
0     000902e4  _App_ServiceMode__13Class_ServiceFv                                                    
0     00089415  _App_SysInitBasedUPSName__12Class_SystemFv                                             
0     00089053  _App_SysInitSunStreaker_208__12Class_SystemFv                                          
0     00089234  _App_SysInitSunStreaker_400__12Class_SystemFv                                          
0     0008955c  _App_SysParamConfig__12Class_SystemFv                                                  
0     00088e8b  _App_SysVarInit__12Class_SystemFv                                                      
0     000115a3  _App_TimeLabel__22Class_MonitorInterfaceFv                                             
0     0008f45e  _App_TraceControl__21Class_InverterControlFv                                           
0     0008f573  _App_TraceJudge__21Class_InverterControlFv                                             
0     0008f415  _App_TraceSignal__21Class_InverterControlFv                                            
0     0008f6cb  _App_XferCommand__14Class_TransferFv                                                   
0     0008ffea  _App_XferExecute__14Class_TransferFv                                                   
0     0008f648  _App_XferOut__14Class_TransferFv                                                       
0     0008fc1c  _App_XferProcess__14Class_TransferFv                                                   
0     000938b4  _BattEodTurnOff__15SysCanDataExchgFv                                                   
0     000938fc  _BattGndPtcCmd__15SysCanDataExchgFv                                                    
0     000938c6  _BattTrip__15SysCanDataExchgFv                                                         
0     00093a64  _BypFPGAFlashUpdate__15SysCanDataExchgFv                                               
0     00093a0c  _BypFlashUpdate__15SysCanDataExchgFv                                                   
0     0009462d  _BypMaintMsgRecvProc__15SysCanDataExchgFP19can_msg_data_struct                         
0     00094bd6  _CANA0_ISR                                                                             
0     00094bdb  _CANA1_ISR                                                                             
0     00094be0  _CANB0_ISR                                                                             
0     00094be5  _CANB1_ISR                                                                             
0     00091f74  _CANDat_MBox_Read__15Class_FPGAFlashFv                                                 
0     00091f78  _CANDat_MBox_Send__15Class_FPGAFlashFUiT1                                              
0     00092a89  _CANFragRecvTimeoutFcb__14SysCanProtocolFv                                             
0     00094c12  _CLA1_1_ISR                                                                            
0     00094c17  _CLA1_2_ISR                                                                            
0     00094c1c  _CLA1_3_ISR                                                                            
0     00094c21  _CLA1_4_ISR                                                                            
0     00094c26  _CLA1_5_ISR                                                                            
0     00094c2b  _CLA1_6_ISR                                                                            
0     00094c30  _CLA1_7_ISR                                                                            
0     00094c35  _CLA1_8_ISR                                                                            
0     00094cdf  _CLA_OVERFLOW_ISR                                                                      
0     00094ce4  _CLA_UNDERFLOW_ISR                                                                     
0     0008714d  _CanFrameTransferToMessage__FP13tCANMsgObjectP9Can_Frame                               
0     0008710d  _CanMessageTransferToFrame__FP9Can_FrameP13tCANMsgObject                               
0     00093aa5  _CfgFragMsgPacked__15SysCanDataExchgFP19can_msg_data_struct                            
0     000934c2  _CfgMsgFromMonProc__15SysCanDataExchgFP19can_msg_data_structUi                         
0     00093cf3  _CfgMsgObjsInit__15SysCanDataExchgFv                                                   
0     000933ce  _CfgMsgRecvProc__15SysCanDataExchgFP19can_msg_data_struct                              
0     0009400b  _CfgMsgRqPacked__15SysCanDataExchgFP19can_msg_data_structi                             
0     0009403a  _CfgMsgRsPacked__15SysCanDataExchgFP19can_msg_data_structi                             
0     000935d3  _CfgMsgToMonProc__15SysCanDataExchgFP19can_msg_data_structUi                           
0     00008300  _Cla1ConstLoadEnd                                                                      
abs   00000000  _Cla1ConstLoadSize                                                                     
0     00008300  _Cla1ConstLoadStart                                                                    
0     00008300  _Cla1ConstRunStart                                                                     
1     00001400  _Cla1Regs                                                                              
0     00000ce0  _Cla1SoftIntRegs                                                                       
0     00008800  _Cla1funcsLoadEnd                                                                      
abs   00000000  _Cla1funcsLoadSize                                                                     
0     00008800  _Cla1funcsLoadStart                                                                    
0     00008800  _Cla1funcsRunStart                                                                     
1     0005d200  _ClkCfgRegs                                                                            
0     000871a2  _CloseSysCanInt__Fv                                                                    
1     00005c80  _Cmpss1Regs                                                                            
1     00005ca0  _Cmpss2Regs                                                                            
1     00005cc0  _Cmpss3Regs                                                                            
1     00005ce0  _Cmpss4Regs                                                                            
1     00005d00  _Cmpss5Regs                                                                            
1     00005d20  _Cmpss6Regs                                                                            
1     00005d40  _Cmpss7Regs                                                                            
1     00005d60  _Cmpss8Regs                                                                            
0     000947af  _CovMsgProc__9SysCanAppFv                                                              
0     00093bbd  _CovSyncMsgObjInit__15SysCanDataExchgFv                                                
1     0005d300  _CpuSysRegs                                                                            
1     00000c00  _CpuTimer0Regs                                                                         
1     00000c08  _CpuTimer1Regs                                                                         
1     00000c10  _CpuTimer2Regs                                                                         
0     00086b40  _CriticalIntFuncsNOTSecuredLoadEnd                                                     
0     00084000  _CriticalIntFuncsNOTSecuredLoadStart                                                   
0     0000f000  _CriticalIntFuncsNOTSecuredRunStart                                                    
0     00097a22  _CriticalIntFuncsSecuredLoadEnd                                                        
0     00097449  _CriticalIntFuncsSecuredLoadStart                                                      
0     0000b050  _CriticalIntFuncsSecuredRunStart                                                       
0     00093b91  _CtrlMsgObjsInit__15SysCanDataExchgFv                                                  
0     0009370c  _CtrlMsgRecvProc__15SysCanDataExchgFP19can_msg_data_struct                             
0     00094a5f  _DATALOG_ISR                                                                           
0     00094b7c  _DMA_CH1_ISR                                                                           
0     00094b81  _DMA_CH2_ISR                                                                           
0     00094b86  _DMA_CH3_ISR                                                                           
0     00094b8b  _DMA_CH4_ISR                                                                           
0     00094b90  _DMA_CH5_ISR                                                                           
0     00094b95  _DMA_CH6_ISR                                                                           
1     00005c00  _DacaRegs                                                                              
1     00005c10  _DacbRegs                                                                              
1     00005c20  _DaccRegs                                                                              
0     0008aa87  _Dat_BoardTypeCheck__15Class_DigitalIOFv                                               
0     0008b437  _Dat_BpRMS__12Class_BypassFv                                                           
0     0008ac3f  _Dat_BreakerStatus__14Class_SwitchesFv                                                 
0     0000b050  _Dat_CRCCalculate__17Class_FlashUpdateFPUiUi                                           
0     0008a103  _Dat_Can_NoyBypCalculation__21Class_PowCANSchedulerFv                                  
0     0008d04e  _Dat_DCBusRMS__11Class_DCBusFv                                                         
0     0008a46d  _Dat_DigitalInput__15Class_DigitalIOFv                                                 
0     0008a9c3  _Dat_DigitalOutput__15Class_DigitalIOFv                                                
0     0008bf61  _Dat_ECOBpFlag__12Class_BypassFv                                                       
0     0009065d  _Dat_EEPROMInit__12Class_EEPROMFv                                                      
0     0008ac10  _Dat_FPGAIDCheck__15Class_DigitalIOFv                                                  
0     0008c3ef  _Dat_IinvRMS__14Class_InverterFv                                                       
0     000114c4  _Dat_Int_DCBusPreDeal__11Class_DCBusFv                                                 
0     000107fa  _Dat_Int_InvCalc2__14Class_InverterFv                                                  
0     00010b1a  _Dat_Int_InvCalc3__14Class_InverterFv                                                  
0     00010b8c  _Dat_Int_InvCurrPQCalc__14Class_InverterFv                                             
0     0001065e  _Dat_Int_InvPreDeal__14Class_InverterFv                                                
0     00011716  _Dat_Int_LBSCapDeal__9Class_LBSFv                                                      
0     000103b7  _Dat_Int_MainInterfaceIn__15Class_DigitalIOFv                                          
0     00010289  _Dat_Int_MainInterfaceOut__15Class_DigitalIOFv                                         
0     00010e24  _Dat_Int_OutCalc2__12Class_OutputFv                                                    
0     00010f36  _Dat_Int_PFDeal__12Class_OutputFv                                                      
0     0008aa7f  _Dat_InvIDOk__15Class_DigitalIOFv                                                      
0     0008e70f  _Dat_LoadDeal__10Class_LoadFv                                                          
0     0008e805  _Dat_LoadFlag__10Class_LoadFv                                                          
0     0008e72f  _Dat_LoadGrant__10Class_LoadFv                                                         
0     0000b0d3  _Dat_MBox_Read__17Class_FlashUpdateFv                                                  
0     0000b25d  _Dat_MBox_Send__17Class_FlashUpdateFUiT1                                               
0     0008ab53  _Dat_ModuleIDGet__15Class_DigitalIOFv                                                  
0     0008ebda  _Dat_OvloadFlag__10Class_LoadFv                                                        
0     0008c5dc  _Dat_PinvRMS__14Class_InverterFv                                                       
0     0008ccc4  _Dat_PoutRMS__12Class_OutputFv                                                         
0     0008a9fc  _Dat_ServiceAndModuleTypeCheck__15Class_DigitalIOFv                                    
0     0008c52c  _Dat_TempPowerGrant__14Class_InverterFv                                                
0     0008b5cb  _Dat_VbpFlag__12Class_BypassFv                                                         
0     0008c769  _Dat_VinvFlag__14Class_InverterFv                                                      
0     0008c270  _Dat_VinvRMS__14Class_InverterFv                                                       
0     0008cb80  _Dat_VoutRMS__12Class_OutputFv                                                         
1     0005f070  _DcsmCommonRegs                                                                        
1     00078000  _DcsmZ1Otp                                                                             
1     0005f000  _DcsmZ1Regs                                                                            
1     00078200  _DcsmZ2Otp                                                                             
1     0005f040  _DcsmZ2Regs                                                                            
0     00090f38  _DebugAckMessage__11Class_DebugFv                                                      
0     00090dde  _DebugComandHandle__11Class_DebugFv                                                    
1     00012f00  _DebugEEPROMBuff                                                                       
1     00012000  _DebugRxBuff                                                                           
0     00092033  _DelQueue__15SysCanRecvQueueFv                                                         
0     000920a0  _DelQueue__15SysCanXmitQueueFv                                                         
0     0009210d  _DelQueue__19SysCanFragXmitQueueFv                                                     
1     0005d000  _DevCfgRegs                                                                            
1     00007980  _DmaClaSrcSelRegs                                                                      
1     00001000  _DmaRegs                                                                               
0     0008806e  _Drv_AdcSetMode__12Class_ADCDrvFUiN21                                                  
0     0000f008  _Drv_ArrayTransmit__12Class_SPIDrvFPUiT1                                               
0     00087aab  _Drv_CANBitRateSet__12Class_CANDrvFUlN21                                               
0     00087a83  _Drv_CANClkSourceSelect__12Class_CANDrvFUlUi                                           
0     00087db0  _Drv_CANDataRegRead__12Class_CANDrvSFPUcPUli                                           
0     00087d21  _Drv_CANDataRegWrite__12Class_CANDrvSFPUcPUli                                          
0     00087b37  _Drv_CANEnable__12Class_CANDrvFUl                                                      
0     00087b33  _Drv_CANFlashFPGAInit__12Class_CANDrvFv                                                
0     00087da6  _Drv_CANGlobalIntClear__12Class_CANDrvFUlT1                                            
0     00087b4a  _Drv_CANGlobalIntDisable__12Class_CANDrvFUlT1                                          
0     00087b40  _Drv_CANGlobalIntEnable__12Class_CANDrvFUlT1                                           
0     00087d7f  _Drv_CANIntClear__12Class_CANDrvFUlT1                                                  
0     00087b26  _Drv_CANIntEnable__12Class_CANDrvFUlT1                                                 
0     00087d3b  _Drv_CANIntStatus__12Class_CANDrvFUl13tCANIntStsReg                                    
0     00087c46  _Drv_CANMessageGet__12Class_CANDrvFUlT1P13tCANMsgObjectb                               
0     00087b55  _Drv_CANMessageSet__12Class_CANDrvFUlT1P13tCANMsgObject11tMsgObjType                   
0     00087dcb  _Drv_CANMsgObjCTLStatusGet__12Class_CANDrvFUlT1                                        
0     00087d56  _Drv_CANStatusGet__12Class_CANDrvFUl10tCANStsReg                                       
0     000886c6  _Drv_CLAMemCopy__12Class_RAMDrvFPUlN21                                                 
0     000880f1  _Drv_CalAdcINL__12Class_ADCDrvFUi                                                      
0     00090f77  _Drv_ConfigStart__16Class_FPGAConfigFv                                                 
0     000885b1  _Drv_DisableDog__17Class_WatchDogDrvFv                                                 
0     000885c0  _Drv_EnableDog__17Class_WatchDogDrvFv                                                  
0     000874fe  _Drv_GPIO_EnableUnbondedIOPullups__13Class_GPIODrvFv                                   
0     000876af  _Drv_GPIO_SetupPinDirection__13Class_GPIODrvFUiT1                                      
0     0008758d  _Drv_GPIO_SetupPinMux__13Class_GPIODrvFUiN21                                           
0     0008761a  _Drv_GPIO_SetupPinOptions__13Class_GPIODrvFUiN21                                       
0     000876df  _Drv_GPIO_SetupPinValue__13Class_GPIODrvFUiT1                                          
0     00087e90  _Drv_I2CPageWrite__12Class_I2CDrvFUiiPUi                                               
0     00087e1a  _Drv_I2CRead__12Class_I2CDrvFUiiPUi                                                    
0     00087e6e  _Drv_I2CWordWrite__12Class_I2CDrvFUiT1                                                 
0     00087ec5  _Drv_I2CWriteAll__12Class_I2CDrvFPUiPiT1                                               
0     00087f3a  _Drv_InitADC__12Class_ADCDrvFv                                                         
0     000879d7  _Drv_InitCANState__12Class_CANDrvFUl                                                   
0     000878f4  _Drv_InitCAN__12Class_CANDrvFv                                                         
0     00088325  _Drv_InitCAP__12Class_CAPDrvFv                                                         
0     00088771  _Drv_InitCMPSS__14Class_CMPSSDrvFv                                                     
0     0008857d  _Drv_InitCpuTimers__12Class_SysDrvFv                                                   
0     0000b000  _Drv_InitFlash__14Class_FlashDrvFv                                                     
0     00087465  _Drv_InitGPIO__13Class_GPIODrvFv                                                       
0     0008754c  _Drv_InitGpioToDefaltValue__13Class_GPIODrvFv                                          
0     00087ded  _Drv_InitI2C__12Class_I2CDrvFv                                                         
0     000885a3  _Drv_InitInterrupts__12Class_SysDrvFv                                                  
0     00088593  _Drv_InitPIE__12Class_SysDrvFv                                                         
0     0008811f  _Drv_InitPWM__12Class_PWMDrvFv                                                         
0     000884a7  _Drv_InitPeripheralClocks__12Class_SysDrvFv                                            
0     000883ca  _Drv_InitPeripherals__12Class_SysDrvFv                                                 
0     00088532  _Drv_InitPieCtrl__12Class_SysDrvFv                                                     
0     00088556  _Drv_InitPieVectTable__12Class_SysDrvFv                                                
0     00087739  _Drv_InitSCI__12Class_SCIDrvFv                                                         
0     00087753  _Drv_InitSPI__12Class_SPIDrvFv                                                         
0     000883fa  _Drv_InitSysPll__12Class_SysDrvFUiN31                                                  
0     000885dc  _Drv_Init__12Class_RAMDrvFv                                                            
0     0000f0dc  _Drv_Int_ClockMaintain__14Class_TimerDrvFv                                             
0     0008858f  _Drv_Int_InterruptFlagClear__12Class_SysDrvFv                                          
0     0000f0bd  _Drv_Int_PWMActive__12Class_PWMDrvFv                                                   
0     0000f0d4  _Drv_Int_PWMInactive__12Class_PWMDrvFv                                                 
0     000885cb  _Drv_KickDog__17Class_WatchDogDrvFv                                                    
0     000886a9  _Drv_MemCopy__12Class_RAMDrvFPUiN21                                                    
0     000885ea  _Drv_RamCheck__12Class_RAMDrvFv                                                        
0     00087892  _Drv_SPIBBlockErase__12Class_SPIDrvFUl                                                 
0     000878e1  _Drv_SPIBEEPROMActionWaitTime__12Class_SPIDrvFUl                                       
0     000878c9  _Drv_SPIBGetWriteStatus__12Class_SPIDrvFv                                              
0     00087809  _Drv_SPIBPageWrite__12Class_SPIDrvFUliPUi                                              
0     00087789  _Drv_SPIBRead__12Class_SPIDrvFUliPUi                                                   
0     0008785b  _Drv_SPIBSectorErase__12Class_SPIDrvFUl                                                
0     000877c7  _Drv_SPIBWordWrite__12Class_SPIDrvFUlUi                                                
0     0008838f  _Drv_SysCtrlInit__12Class_SysDrvFv                                                     
0     0008847e  _Drv_SysIntOsc1Sel__12Class_SysDrvFv                                                   
0     0008848b  _Drv_SysIntOsc2Sel__12Class_SysDrvFv                                                   
0     000886d9  _Drv_SysTimer__14Class_TimerDrvFv                                                      
0     00088498  _Drv_SysXtalOscSel__12Class_SysDrvFv                                                   
0     00088758  _Drv_usDelay__14Class_TimerDrvFl                                                       
0     00094cf8  _ECAN0INTA_ISR__Fv                                                                     
0     00094b27  _ECAP1_ISR                                                                             
0     00094b2c  _ECAP2_ISR                                                                             
0     00094b31  _ECAP3_ISR                                                                             
0     00094b36  _ECAP4_ISR                                                                             
0     00094b3b  _ECAP5_ISR                                                                             
0     00094b40  _ECAP6_ISR                                                                             
1     00005000  _ECap1Regs                                                                             
1     00005020  _ECap2Regs                                                                             
1     00005040  _ECap3Regs                                                                             
1     00005060  _ECap4Regs                                                                             
1     00005080  _ECap5Regs                                                                             
1     000050a0  _ECap6Regs                                                                             
0     00094cc1  _EMIF_ERROR_ISR                                                                        
0     00094cee  _EMPTY_ISR                                                                             
0     00094a69  _EMU_ISR                                                                               
0     00094c85  _EPWM10_ISR                                                                            
0     00094c71  _EPWM10_TZ_ISR                                                                         
0     00094c8a  _EPWM11_ISR                                                                            
0     00094c76  _EPWM11_TZ_ISR                                                                         
0     00094c8f  _EPWM12_ISR                                                                            
0     00094c7b  _EPWM12_TZ_ISR                                                                         
0     00094aff  _EPWM1_ISR                                                                             
0     00094ad7  _EPWM1_TZ_ISR                                                                          
0     00094b04  _EPWM2_ISR                                                                             
0     00094adc  _EPWM2_TZ_ISR                                                                          
0     00094b09  _EPWM3_ISR                                                                             
0     00094ae1  _EPWM3_TZ_ISR                                                                          
0     00094b0e  _EPWM4_ISR                                                                             
0     00094ae6  _EPWM4_TZ_ISR                                                                          
0     00094b13  _EPWM5_ISR                                                                             
0     00094aeb  _EPWM5_TZ_ISR                                                                          
0     00094b18  _EPWM6_ISR                                                                             
0     00094af0  _EPWM6_TZ_ISR                                                                          
0     00094b1d  _EPWM7_ISR                                                                             
0     00094af5  _EPWM7_TZ_ISR                                                                          
0     00094b22  _EPWM8_ISR                                                                             
0     00094afa  _EPWM8_TZ_ISR                                                                          
0     00094c80  _EPWM9_ISR                                                                             
0     00094c6c  _EPWM9_TZ_ISR                                                                          
0     0000b444  _EPWM_INT_ISR__Fv                                                                      
1     00004900  _EPwm10Regs                                                                            
1     00004a00  _EPwm11Regs                                                                            
1     00004b00  _EPwm12Regs                                                                            
1     00004000  _EPwm1Regs                                                                             
1     00004100  _EPwm2Regs                                                                             
1     00004200  _EPwm3Regs                                                                             
1     00004300  _EPwm4Regs                                                                             
1     00004400  _EPwm5Regs                                                                             
1     00004500  _EPwm6Regs                                                                             
1     00004600  _EPwm7Regs                                                                             
1     00004700  _EPwm8Regs                                                                             
1     00004800  _EPwm9Regs                                                                             
1     00007a00  _EPwmXbarRegs                                                                          
0     00094b45  _EQEP1_ISR                                                                             
0     00094b4a  _EQEP2_ISR                                                                             
0     00094b4f  _EQEP3_ISR                                                                             
1     00005100  _EQep1Regs                                                                             
1     00005140  _EQep2Regs                                                                             
1     00005180  _EQep3Regs                                                                             
1     0005f480  _Emif1ConfigRegs                                                                       
1     00047000  _Emif1Regs                                                                             
1     00000d01  _EmuBMode                                                                              
1     00000d00  _EmuKey                                                                                
0     000940b8  _EndResendTimer__15SysCanDataExchgFv                                                   
0     0009397a  _EpoCmd__15SysCanDataExchgFv                                                           
0     00091f9e  _Excute__14ProtocolSubCmdFPv                                                           
0     000949e4  _Excute__30TemplateCmd__tm__11_9SysCanAppFPv_i                                         
0     00091fd9  _Excute__9AppSubCmdFPv                                                                 
0     0000b625  _F28x_usDelay                                                                          
0     00094ccb  _FLASH_CORRECTABLE_ERROR_ISR                                                           
1     00012000  _FPGACodeEEPROMBuff                                                                    
0     00094c4e  _FPU_OVERFLOW_ISR                                                                      
0     00094c53  _FPU_UNDERFLOW_ISR                                                                     
0     0009390e  _FaultClrCmd__15SysCanDataExchgFv                                                      
0     000948d6  _FaultDataXimt__9SysCanAppFv                                                           
0     00094565  _FaultFragMsgPacked__15SysCanDataExchgFP19can_msg_data_struct                          
0     0000b26d  _FlagProgram__17Class_FlashUpdateFv                                                    
0     0009204b  _FlagQueue__15SysCanRecvQueueFv                                                        
0     000920b8  _FlagQueue__15SysCanXmitQueueFv                                                        
0     00092125  _FlagQueue__19SysCanFragXmitQueueFv                                                    
1     0005f800  _Flash0CtrlRegs                                                                        
1     0005fb00  _Flash0EccRegs                                                                         
0     00081243  _Flash28_API_LoadEnd                                                                   
0     00081000  _Flash28_API_LoadStart                                                                 
0     0000b050  _Flash28_API_RunStart                                                                  
1     00012400  _FlashBuffer                                                                           
0     00092a05  _FragAckTimeoutFcb__14SysCanProtocolFv                                                 
0     00093a84  _FragMsgPacked__15SysCanDataExchgFP19can_msg_data_struct                               
0     00094976  _FragMsgPost__9SysCanAppFv                                                             
0     00092750  _FragMsgRecvStateMachine__14SysCanProtocolFP26CAN_PACKED_PROTOCOL_STRUCT               
0     00092522  _FragMsgXmitStateMachineEnty__14SysCanProtocolFv                                       
0     0009255a  _FragMsgXmitStateMachine__14SysCanProtocolFP26CAN_PACKED_PROTOCOL_STRUCT               
0     000949d4  _FragRecvOkHandle__9SysCanAppFPv                                                       
0     00092a47  _FragXmitBusyTimeoutFcb__14SysCanProtocolFv                                            
0     000949be  _FragXmitErrHandle__9SysCanAppFPv                                                      
0     000949a5  _FragXmitOkHandle__9SysCanAppFPv                                                       
0     00093a72  _FragXmitResult__15SysCanDataExchgFP19can_msg_data_structi                             
0     0009242e  _FrameParseToApdu__14SysCanProtocolFP19can_msg_data_structP26CAN_PACKED_PROTOCOL_STRUCT
0     0009249f  _FrameParseToPpdu__14SysCanProtocolFP26CAN_PACKED_PROTOCOL_STRUCTP19can_msg_data_struct
0     000942a0  _GenAlarmEvent__15SysCanDataExchgFv                                                    
0     000940c9  _GenStateEvent__15SysCanDataExchgFv                                                    
0     00092df4  _GetAlrmCovMsg__15SysCanDataExchgFP19can_msg_data_struct                               
0     00093260  _GetAlrmSyncMsg__15SysCanDataExchgFP19can_msg_data_struct                              
0     000932bb  _GetAnalogSyncMsg__15SysCanDataExchgFP19can_msg_data_struct                            
0     00092d0c  _GetDataExchgPtr__15SysCanDataExchgSFv                                                 
0     00092eb9  _GetEventLogMsg__15SysCanDataExchgFP19can_msg_data_struct                              
0     00093b34  _GetFaultData__15SysCanDataExchgFP19can_msg_data_struct                                
0     0009205d  _GetOldestNode__15SysCanRecvQueueFv                                                    
0     000920ca  _GetOldestNode__15SysCanXmitQueueFv                                                    
0     00092137  _GetOldestNode__19SysCanFragXmitQueueFv                                                
0     00093090  _GetParallelStateMsg__15SysCanDataExchgFP19can_msg_data_struct                         
0     0009408a  _GetResendSysSetFlag__15SysCanDataExchgFv                                              
0     00092d33  _GetStateCovMsg__15SysCanDataExchgFP19can_msg_data_struct                              
0     000931d5  _GetStateSyncMsg__15SysCanDataExchgFP19can_msg_data_struct                             
0     00094679  _GetSyncMonitorCnt__15SysCanDataExchgFv                                                
1     00007c00  _GpioCtrlRegs                                                                          
1     00007f00  _GpioDataRegs                                                                          
0     00094b9f  _I2CA_FIFO_ISR                                                                         
0     00094b9a  _I2CA_ISR                                                                              
0     00094ba9  _I2CB_FIFO_ISR                                                                         
0     00094ba4  _I2CB_ISR                                                                              
1     00007300  _I2caRegs                                                                              
1     00007340  _I2cbRegs                                                                              
0     00094a73  _ILLEGAL_ISR                                                                           
0     00094c58  _IPC0_ISR                                                                              
0     00094c5d  _IPC1_ISR                                                                              
0     00094c62  _IPC2_ISR                                                                              
0     00094c67  _IPC3_ISR                                                                              
0     000939b0  _IndirectSwitchCmd__15SysCanDataExchgFv                                                
0     0008770d  _InitECap1Gpio__13Class_GPIODrvFUi                                                     
0     00087718  _InitECap2Gpio__13Class_GPIODrvFUi                                                     
0     00087723  _InitECap3Gpio__13Class_GPIODrvFUi                                                     
0     0008772e  _InitECap4Gpio__13Class_GPIODrvFUi                                                     
1     00007900  _InputXbarRegs                                                                         
0     0009200a  _InsQueue__15SysCanRecvQueueF26CAN_PACKED_PROTOCOL_STRUCT                              
0     00092077  _InsQueue__15SysCanXmitQueueF26CAN_PACKED_PROTOCOL_STRUCT                              
0     000920e4  _InsQueue__19SysCanFragXmitQueueF19can_msg_data_struct                                 
0     00092ae6  _InterfaceDataProc__15SysCanDataExchgFv                                                
0     00093a30  _InvFPGAFlashUpdate__15SysCanDataExchgFv                                               
0     000939d8  _InvFlashUpdate__15SysCanDataExchgFv                                                   
0     00094b68  _MCBSPA_RX_ISR                                                                         
0     00094b6d  _MCBSPA_TX_ISR                                                                         
0     00094b72  _MCBSPB_RX_ISR                                                                         
0     00094b77  _MCBSPB_TX_ISR                                                                         
0     0009473c  _MainRoutie__9SysCanAppFv                                                              
0     000945b5  _MaintParallelData__15SysCanDataExchgFv                                                
0     00093954  _MaualShutCmd__15SysCanDataExchgFv                                                     
0     0009392e  _MaualStartupCmd__15SysCanDataExchgFv                                                  
1     00006000  _McbspaRegs                                                                            
1     00006040  _McbspbRegs                                                                            
1     0005f400  _MemCfgRegs                                                                            
1     0005f500  _MemoryErrorRegs                                                                       
0     000946a9  _MonRealMsgRecvProc__15SysCanDataExchgFP19can_msg_data_struct                          
0     000946cc  _MonitorCanErrDetect__15SysCanDataExchgFv                                              
0     00093386  _MonitorSyncMsgProc__15SysCanDataExchgFv                                               
0     00092332  _MsgRecvProc__14SysCanProtocolFP19can_msg_data_struct                                  
0     00094711  _MsgRecvProc__9SysCanAppFv                                                             
0     00092392  _MsgXmitProc__14SysCanProtocolFP19can_msg_data_struct                                  
0     00094a6e  _NMI_ISR                                                                               
0     00094cf3  _NOTUSED_ISR                                                                           
1     00007060  _NmiIntruptRegs                                                                        
0     000871b8  _OpenSysCanInt__Fv                                                                     
0     000938ea  _OutputDisableCmd__15SysCanDataExchgFv                                                 
0     000938d8  _OutputEnableCmd__15SysCanDataExchgFv                                                  
1     00007a80  _OutputXbarRegs                                                                        
0     00094ce9  _PIE_RESERVED_ISR                                                                      
0     00094a12  _PIE_RESERVED__Fv                                                                      
0     0009458e  _ParallelMsgRecvProc__15SysCanDataExchgFP19can_msg_data_struct                         
0     000930cb  _ParallelStateXmitMsgGen__15SysCanDataExchgFUi                                         
0     00093320  _PeriodAnalogSyncMsg__15SysCanDataExchgFP19can_msg_data_struct                         
0     00093def  _PeriodPowerXmitMsgGen__15SysCanDataExchgFUi                                           
1     00000ce0  _PieCtrlRegs                                                                           
1     00000d00  _PieVectTable                                                                          
0     00094cd0  _RAM_ACCESS_VIOLATION_ISR                                                              
0     00094cc6  _RAM_CORRECTABLE_ERROR_ISR                                                             
0     00094a64  _RTOS_ISR                                                                              
0     00094650  _RackStateMsgRecvProc__15SysCanDataExchgFP19can_msg_data_struct                        
0     000953b8  _RamfuncsLoadEnd                                                                       
abs   00000028  _RamfuncsLoadSize                                                                      
0     00095390  _RamfuncsLoadStart                                                                     
0     0000b028  _RamfuncsRunEnd                                                                        
abs   00000028  _RamfuncsRunSize                                                                       
0     0000b000  _RamfuncsRunStart                                                                      
0     00093a22  _RecFPGAFlashUpdate__15SysCanDataExchgFv                                               
0     000939c2  _RecFlashUpdate__15SysCanDataExchgFv                                                   
1     0000c034  _ReceiveFrame                                                                          
0     0009490c  _RecvMsgDispatch__9SysCanAppFP19can_msg_data_struct                                    
0     00092f35  _ReqSetMsg__15SysCanDataExchgFP19can_msg_data_struct                                   
0     000940a8  _RestartResendTimer__15SysCanDataExchgFv                                               
1     0005e608  _RomPrefetchRegs                                                                       
1     0005f540  _RomWaitStateRegs                                                                      
0     00094bc2  _SCIA_RX_ISR                                                                           
0     00094bc7  _SCIA_TX_ISR                                                                           
0     00094bcc  _SCIB_RX_ISR                                                                           
0     00094bd1  _SCIB_TX_ISR                                                                           
0     00094bae  _SCIC_RX_ISR                                                                           
0     00094bb3  _SCIC_TX_ISR                                                                           
0     00094bb8  _SCID_RX_ISR                                                                           
0     00094bbd  _SCID_TX_ISR                                                                           
0     000119fb  _SCI_ReceiveEnd__15Class_FPGAFlashFv                                                   
0     00094c94  _SD1_ISR                                                                               
0     00094c99  _SD2_ISR                                                                               
0     00094b54  _SPIA_RX_ISR                                                                           
0     00094b59  _SPIA_TX_ISR                                                                           
0     00094b5e  _SPIB_RX_ISR                                                                           
0     00094b63  _SPIB_TX_ISR                                                                           
0     00094c9e  _SPIC_RX_ISR                                                                           
0     00094ca3  _SPIC_TX_ISR                                                                           
0     00094cd5  _SYS_PLL_SLIP_ISR                                                                      
0     00091c65  _SciFrameOverTime__15Class_FPGAFlashFv                                                 
1     00007200  _SciaRegs                                                                              
1     00007210  _ScibRegs                                                                              
1     00007220  _ScicRegs                                                                              
1     00007230  _ScidRegs                                                                              
1     00005e00  _Sdfm1Regs                                                                             
1     00005e80  _Sdfm2Regs                                                                             
0     000923c7  _SetFragRecvOkHandleFcb__14SysCanProtocolFP11CommandBase                               
0     000923e3  _SetFragXmitErrHandleFcb__14SysCanProtocolFP11CommandBase                              
0     000923fd  _SetFragXmitOkHandleFcb__14SysCanProtocolFP11CommandBase                               
1     00006100  _SpiaRegs                                                                              
1     00006110  _SpibRegs                                                                              
1     00006120  _SpicRegs                                                                              
0     00092d6a  _StateCovMsgXmitState__15SysCanDataExchgFi                                             
0     00093017  _StateEventXmitMsgGen__15SysCanDataExchgFUi                                            
0     00093433  _StateMsgRecvProc__15SysCanDataExchgFP19can_msg_data_struct                            
0     00093251  _StateSyncMsgXmitState__15SysCanDataExchgFi                                            
0     00092d79  _StateXmitMsgGen__15SysCanDataExchgFUi                                                 
0     00093147  _SyncFlagDelayProc__15SysCanDataExchgFP19can_msg_data_struct                           
0     00093471  _SyncMsgProc__15SysCanDataExchgFP19can_msg_data_struct                                 
0     0009483a  _SyncMsgProc__9SysCanAppFv                                                             
1     00007940  _SyncSocRegs                                                                           
0     00093670  _SyncTimeMsgProc__15SysCanDataExchgFP19can_msg_data_struct                             
0     00092acc  _SysCanDataExchgIni__15SysCanDataExchgFv                                               
0     000870f8  _SysCanFcbRegister__FP11CommandBaseT1                                                  
0     000920d8  _SysCanFragXmitQueueIni__19SysCanFragXmitQueueFv                                       
0     0009475a  _SysCanInitial__9SysCanAppFv                                                           
0     00092145  _SysCanProtocolIni__14SysCanProtocolFv                                                 
0     00092254  _SysCanRecvFcb__14SysCanProtocolFPv                                                    
0     00091ffe  _SysCanRecvQueueIni__15SysCanRecvQueueFv                                               
0     000871c4  _SysCanSendData__FP9Can_Frame                                                          
0     0009229c  _SysCanXmitFcb__14SysCanProtocolFPv                                                    
0     0009206b  _SysCanXmitQueueIni__15SysCanXmitQueueFv                                               
0     00094acd  _TIMER0_ISR                                                                            
0     00094a55  _TIMER1_ISR                                                                            
0     00094a5a  _TIMER2_ISR                                                                            
0     00092417  _Timer_Expire_Handle__14SysCanProtocolFv                                               
0     00092abb  _Timer_Flush__14SysCanProtocolFP14TIMER_HANDLE_T                                       
0     00092aa5  _Timer_Post__14SysCanProtocolFP14TIMER_HANDLE_T                                        
0     00094ca8  _USBA_ISR                                                                              
0     00094aa5  _USER10_ISR                                                                            
0     00094aaa  _USER11_ISR                                                                            
0     00094aaf  _USER12_ISR                                                                            
0     00094a78  _USER1_ISR                                                                             
0     00094a7d  _USER2_ISR                                                                             
0     00094a82  _USER3_ISR                                                                             
0     00094a87  _USER4_ISR                                                                             
0     00094a8c  _USER5_ISR                                                                             
0     00094a91  _USER6_ISR                                                                             
0     00094a96  _USER7_ISR                                                                             
0     00094a9b  _USER8_ISR                                                                             
0     00094aa0  _USER9_ISR                                                                             
0     00094c49  _VCU_ISR                                                                               
0     00091c13  _VarReset__15Class_FPGAFlashFv                                                         
0     00094ad2  _WAKE_ISR                                                                              
1     00007000  _WdRegs                                                                                
0     00094abe  _XINT1_ISR                                                                             
0     00094ac3  _XINT2_ISR                                                                             
0     00094c3a  _XINT3_ISR                                                                             
0     00094c3f  _XINT4_ISR                                                                             
0     00094c44  _XINT5_ISR                                                                             
1     00007920  _XbarRegs                                                                              
1     00007070  _XintRegs                                                                              
0     000922d9  _XmitFramePost__14SysCanProtocolFP26CAN_PACKED_PROTOCOL_STRUCT                         
1     00000600  __STACK_END                                                                            
abs   00000200  __STACK_SIZE                                                                           
abs   00000400  __SYSMEM_SIZE                                                                          
0     00091f88  ___CPR75__ProtocolSubCmdIni__14ProtocolSubCmdFP14SysCanProtocolMJ37JFPv_i              
1     0000d9b8  ___TI_cleanup_ptr                                                                      
1     0000d9ba  ___TI_dtors_ptr                                                                        
1     0000d9b6  ___TI_enable_exit_profile_output                                                       
abs   ffffffff  ___TI_pprof_out_hndl                                                                   
abs   ffffffff  ___TI_prof_data_size                                                                   
abs   ffffffff  ___TI_prof_data_start                                                                  
0     00095388  ___abort_execution                                                                     
0     00095282  ___add_dtor                                                                            
1     0000d9c1  ___atexit_func_id__                                                                    
abs   ffffffff  ___binit__                                                                             
abs   ffffffff  ___c_args__                                                                            
0     00097a24  ___cinit__                                                                             
0     0009538d  ___default_new_handler__Fv                                                             
0     0009537f  ___dl__FPv                                                                             
0     0009538f  ___etext__                                                                             
0     000952d3  ___nw__FUl                                                                             
0     00097abc  ___pinit__                                                                             
0     00095384  ___pure_virtual_called                                                                 
0     00094a09  ___sti___17_MainProcedure_cpp_6cdd801d                                                 
0     00086b40  ___text__                                                                              
0     00097402  ___vtbl__14ProtocolSubCmd                                                              
0     0009740e  ___vtbl__30TemplateCmd__tm__11_9SysCanApp                                              
0     0009532a  __args_main                                                                            
1     0000d9bc  __lock                                                                                 
1     0000dac2  __new_handler                                                                          
0     00095376  __nop                                                                                  
0     00095372  __register_lock                                                                        
0     0009536e  __register_unlock                                                                      
1     00000400  __stack                                                                                
1     0000e800  __sys_memory                                                                           
0     0009538e  __system_post_cinit                                                                    
0     0009538b  __system_pre_init                                                                      
1     0000d9be  __unlock                                                                               
0     0009521a  _abort                                                                                 
1     000121c0  _byCRCHiArrayFlash                                                                     
1     000120c0  _byCRCLoArrayFlash                                                                     
0     0009519c  _c_int00                                                                               
0     00011990  _cal_sumcheck__11Class_DebugFPUiUi                                                     
0     00091bc0  _cal_sumcheck__15Class_FPGAFlashFPUiUi                                                 
0     00094fa1  _calloc                                                                                
0     00094f9f  _chkheap                                                                               
0     00094db1  _cla1Isr1__Fv                                                                          
0     00094dbe  _cla1Isr2__Fv                                                                          
0     00094dc4  _cla1Isr3__Fv                                                                          
0     00094dca  _cla1Isr4__Fv                                                                          
0     00094dd0  _cla1Isr5__Fv                                                                          
0     00094dd6  _cla1Isr6__Fv                                                                          
0     00094ddc  _cla1Isr7__Fv                                                                          
0     00094de2  _cla1Isr8__Fv                                                                          
0     0009528d  _copy_in                                                                               
0     0009521c  _exit                                                                                  
0     00094deb  _free                                                                                  
0     00094f84  _free_memory                                                                           
1     0000c022  _g_bErrFlag                                                                            
1     0000c00f  _g_i16_IntCnt1Per2_0                                                                   
1     0000c00e  _g_i16_IntCnt1Per4_0                                                                   
1     0000c00b  _g_u16_INTRunTime                                                                      
1     0000c00d  _g_u16_INTRunTimeMax                                                                   
1     0000c013  _g_u16_MainRunTime                                                                     
1     0000c00c  _g_u16_MainRunTimeMax                                                                  
1     0000c020  _g_ulRxMsgCount                                                                        
1     0000c024  _g_ulTxMsgCount                                                                        
0     00087093  _igap__FiPC10FLAG_TABLET1                                                              
1     0000c01c  _m_pDataExchgPtr__15SysCanDataExchg                                                    
1     000122c0  _m_u16_SCIRxBuff                                                                       
0     000871e4  _main                                                                                  
0     00094e54  _malloc                                                                                
0     00094f65  _max_free                                                                              
0     000952f3  _memcpy                                                                                
0     00095357  _memset                                                                                
0     00094e31  _minit                                                                                 
1     0000c1c0  _objADCDrv                                                                             
1     0000c340  _objBypass                                                                             
1     0000c006  _objCANDrv                                                                             
1     0000c009  _objCAPDrv                                                                             
1     0000c005  _objCLA                                                                                
1     0000c003  _objCMPSSDrv                                                                           
1     0000c0ac  _objDCBus                                                                              
1     0000cf80  _objDataExchg                                                                          
1     0000c280  _objDebug                                                                              
1     0000c2c0  _objDigitalIO                                                                          
1     0000c012  _objECO                                                                                
1     0000c180  _objEEPROM                                                                             
1     0000c02a  _objFPGAConfig                                                                         
1     0000c840  _objFPGAFlash                                                                          
1     0000c026  _objFaultRecord                                                                        
1     0000c008  _objFlashDrv                                                                           
1     0000c011  _objFlashUpdate                                                                        
1     0000c00a  _objGPIODrv                                                                            
1     0000c007  _objI2CDrv                                                                             
1     0000c480  _objInvAlg                                                                             
1     0000c0cf  _objInvCtrl                                                                            
1     0000d340  _objInverter                                                                           
1     0000c09e  _objLBS                                                                                
1     0000c200  _objLoad                                                                               
1     0000c600  _objMonInterface                                                                       
1     0000c3c0  _objOutput                                                                             
1     0000c001  _objPWMDrv                                                                             
1     0000c040  _objParallel                                                                           
1     0000c010  _objPowCANPro                                                                          
1     0000ca40  _objPowCANSched                                                                        
1     0000cc80  _objProtocol                                                                           
1     0000c000  _objRAMDrv                                                                             
1     0000c002  _objSCIDrv                                                                             
1     0000c100  _objSPIDrv                                                                             
1     0000c240  _objSelfAgingAlg                                                                       
1     0000c015  _objService                                                                            
1     0000c0c0  _objSwitches                                                                           
1     0000c700  _objSysCanApp                                                                          
1     0000c017  _objSysDrv                                                                             
1     0000c540  _objSystem                                                                             
1     0000c067  _objTimerDrv                                                                           
1     0000c004  _objWatchDogDrv                                                                        
1     0000c140  _objXfer                                                                               
1     0000c01e  _pCanIsrRecvFcb                                                                        
1     0000c01a  _pCanIsrXmitFcb                                                                        
0     00094eb1  _realloc                                                                               
1     0000c08a  _sRXCANAMessage                                                                        
1     0000c080  _sRXCANBMessage                                                                        
1     0000c070  _sTXCANAMessage                                                                        
1     0000c094  _sTXCANBMessage                                                                        
1     00012800  _st_FlashVariable                                                                      
1     00012080  _u16FaultRecordRead                                                                    
1     0000c014  _u16_FPGA_Flash_CANInit                                                                
1     00012000  _uFaultRecord                                                                          
1     00012100  _uFaultRecordBuff                                                                      
1     0000c0de  _uInvAnalogLen                                                                         
1     0000c047  _ucRXAMsgData                                                                          
1     0000c057  _ucRXBMsgData                                                                          
1     0000c04f  _ucTXAMsgData                                                                          
1     0000c05f  _ucTXBMsgData                                                                          
0     00091be2  _wCRC__15Class_FPGAFlashFPUiUi                                                         
abs   ffffffff  binit                                                                                  
0     00097a24  cinit                                                                                  
0     00080000  code_start                                                                             
0     0009538f  etext                                                                                  
0     00097abc  pinit                                                                                  


GLOBAL SYMBOLS: SORTED BY Symbol Address 

page  address   name                                                                                   
----  -------   ----                                                                                   
0     00000ce0  _Cla1SoftIntRegs                                                                       
0     00008300  _Cla1ConstLoadEnd                                                                      
0     00008300  _Cla1ConstLoadStart                                                                    
0     00008300  _Cla1ConstRunStart                                                                     
0     00008800  _Cla1funcsLoadEnd                                                                      
0     00008800  _Cla1funcsLoadStart                                                                    
0     00008800  _Cla1funcsRunStart                                                                     
0     0000b000  _Drv_InitFlash__14Class_FlashDrvFv                                                     
0     0000b000  _RamfuncsRunStart                                                                      
0     0000b028  _RamfuncsRunEnd                                                                        
0     0000b050  _CriticalIntFuncsSecuredRunStart                                                       
0     0000b050  _Dat_CRCCalculate__17Class_FlashUpdateFPUiUi                                           
0     0000b050  _Flash28_API_RunStart                                                                  
0     0000b081  _App_FlashAPIInit__17Class_FlashUpdateFv                                               
0     0000b08f  _App_FlashUpdateMain__17Class_FlashUpdateFv                                            
0     0000b093  _App_Flash_CsmUnlock__17Class_FlashUpdateFv                                            
0     0000b0a1  _App_Delay1ms__17Class_FlashUpdateFv                                                   
0     0000b0ba  _App_Delay20ms__17Class_FlashUpdateFv                                                  
0     0000b0d3  _Dat_MBox_Read__17Class_FlashUpdateFv                                                  
0     0000b25d  _Dat_MBox_Send__17Class_FlashUpdateFUiT1                                               
0     0000b263  _App_DSPRestart__17Class_FlashUpdateFv                                                 
0     0000b26d  _FlagProgram__17Class_FlashUpdateFv                                                    
0     0000b444  _EPWM_INT_ISR__Fv                                                                      
0     0000b625  _F28x_usDelay                                                                          
0     0000f000  _CriticalIntFuncsNOTSecuredRunStart                                                    
0     0000f008  _Drv_ArrayTransmit__12Class_SPIDrvFPUiT1                                               
0     0000f0bd  _Drv_Int_PWMActive__12Class_PWMDrvFv                                                   
0     0000f0d4  _Drv_Int_PWMInactive__12Class_PWMDrvFv                                                 
0     0000f0dc  _Drv_Int_ClockMaintain__14Class_TimerDrvFv                                             
0     0000f102  _Alg_Int_InvOffReset__23Class_InverterAlgorithmFv                                      
0     0000f176  _Alg_Int_CarrierPowerCANSync__23Class_InverterAlgorithmFv                              
0     0000f285  _Alg_Int_PhaseLock1__23Class_InverterAlgorithmFv                                       
0     0000f8b0  _Alg_Int_InvSyncPulseGen__23Class_InverterAlgorithmFv                                  
0     0000f9c1  _Alg_Int_InvSyncPulseRec__23Class_InverterAlgorithmFv                                  
0     0000fa86  _Alg_Int_InvSyncRecord__23Class_InverterAlgorithmFv                                    
0     0000fa98  _Alg_Int_LockStatus__23Class_InverterAlgorithmFv                                       
0     0000fc22  _Alg_Int_ECOFreqFastChk__23Class_InverterAlgorithmFv                                   
0     0000fcb1  _App_Int_CurrSharOptPreDeal_Route1__21Class_PowCANSchedulerFv                          
0     00010262  _App_Int_Can_SendSchedule__21Class_PowCANSchedulerFv                                   
0     00010289  _Dat_Int_MainInterfaceOut__15Class_DigitalIOFv                                         
0     000103b7  _Dat_Int_MainInterfaceIn__15Class_DigitalIOFv                                          
0     00010542  _App_Int_SPIAct__15Class_DigitalIOFv                                                   
0     0001059d  _Alg_Int_STSDiffFastChk__14Class_SwitchesFv                                            
0     0001065e  _Dat_Int_InvPreDeal__14Class_InverterFv                                                
0     000107fa  _Dat_Int_InvCalc2__14Class_InverterFv                                                  
0     00010b1a  _Dat_Int_InvCalc3__14Class_InverterFv                                                  
0     00010b8c  _Dat_Int_InvCurrPQCalc__14Class_InverterFv                                             
0     00010d21  _App_Int_InvOffReset__14Class_InverterFv                                               
0     00010e24  _Dat_Int_OutCalc2__12Class_OutputFv                                                    
0     00010f36  _Dat_Int_PFDeal__12Class_OutputFv                                                      
0     00010f3a  _Alg_Int_VoutFastChk__12Class_OutputFv                                                 
0     00011327  _Alg_Int_VoutAbnormal__12Class_OutputFv                                                
0     000114c4  _Dat_Int_DCBusPreDeal__11Class_DCBusFv                                                 
0     000114ed  _Alg_Int_DCOVProtect__11Class_DCBusFv                                                  
0     000115a3  _App_TimeLabel__22Class_MonitorInterfaceFv                                             
0     000115ee  _App_Int_ECOInvSoftstart__21Class_InverterControlFv                                    
0     0001167d  _App_Int_FlagCntReset__21Class_InverterControlFv                                       
0     00011716  _Dat_Int_LBSCapDeal__9Class_LBSFv                                                      
0     00011765  _Alg_Int_LBSDetect__9Class_LBSFv                                                       
0     0001178f  _App_Int_WaveRecord__11Class_DebugFv                                                   
0     00011990  _cal_sumcheck__11Class_DebugFPUiUi                                                     
0     000119a9  _App_Int_VirtualScopeStartup__11Class_DebugFv                                          
0     000119fb  _SCI_ReceiveEnd__15Class_FPGAFlashFv                                                   
0     00011a62  _App_Int_SciFrameReceive__15Class_FPGAFlashFv                                          
0     00080000  code_start                                                                             
0     00081000  _Flash28_API_LoadStart                                                                 
0     00081243  _Flash28_API_LoadEnd                                                                   
0     00084000  _CriticalIntFuncsNOTSecuredLoadStart                                                   
0     00086b40  .text                                                                                  
0     00086b40  _CriticalIntFuncsNOTSecuredLoadEnd                                                     
0     00086b40  ___text__                                                                              
0     00087093  _igap__FiPC10FLAG_TABLET1                                                              
0     000870f8  _SysCanFcbRegister__FP11CommandBaseT1                                                  
0     0008710d  _CanMessageTransferToFrame__FP9Can_FrameP13tCANMsgObject                               
0     0008714d  _CanFrameTransferToMessage__FP13tCANMsgObjectP9Can_Frame                               
0     000871a2  _CloseSysCanInt__Fv                                                                    
0     000871b8  _OpenSysCanInt__Fv                                                                     
0     000871c4  _SysCanSendData__FP9Can_Frame                                                          
0     000871e4  _main                                                                                  
0     00087465  _Drv_InitGPIO__13Class_GPIODrvFv                                                       
0     000874fe  _Drv_GPIO_EnableUnbondedIOPullups__13Class_GPIODrvFv                                   
0     0008754c  _Drv_InitGpioToDefaltValue__13Class_GPIODrvFv                                          
0     0008758d  _Drv_GPIO_SetupPinMux__13Class_GPIODrvFUiN21                                           
0     0008761a  _Drv_GPIO_SetupPinOptions__13Class_GPIODrvFUiN21                                       
0     000876af  _Drv_GPIO_SetupPinDirection__13Class_GPIODrvFUiT1                                      
0     000876df  _Drv_GPIO_SetupPinValue__13Class_GPIODrvFUiT1                                          
0     0008770d  _InitECap1Gpio__13Class_GPIODrvFUi                                                     
0     00087718  _InitECap2Gpio__13Class_GPIODrvFUi                                                     
0     00087723  _InitECap3Gpio__13Class_GPIODrvFUi                                                     
0     0008772e  _InitECap4Gpio__13Class_GPIODrvFUi                                                     
0     00087739  _Drv_InitSCI__12Class_SCIDrvFv                                                         
0     00087753  _Drv_InitSPI__12Class_SPIDrvFv                                                         
0     00087789  _Drv_SPIBRead__12Class_SPIDrvFUliPUi                                                   
0     000877c7  _Drv_SPIBWordWrite__12Class_SPIDrvFUlUi                                                
0     00087809  _Drv_SPIBPageWrite__12Class_SPIDrvFUliPUi                                              
0     0008785b  _Drv_SPIBSectorErase__12Class_SPIDrvFUl                                                
0     00087892  _Drv_SPIBBlockErase__12Class_SPIDrvFUl                                                 
0     000878c9  _Drv_SPIBGetWriteStatus__12Class_SPIDrvFv                                              
0     000878e1  _Drv_SPIBEEPROMActionWaitTime__12Class_SPIDrvFUl                                       
0     000878f4  _Drv_InitCAN__12Class_CANDrvFv                                                         
0     000879d7  _Drv_InitCANState__12Class_CANDrvFUl                                                   
0     00087a83  _Drv_CANClkSourceSelect__12Class_CANDrvFUlUi                                           
0     00087aab  _Drv_CANBitRateSet__12Class_CANDrvFUlN21                                               
0     00087b26  _Drv_CANIntEnable__12Class_CANDrvFUlT1                                                 
0     00087b33  _Drv_CANFlashFPGAInit__12Class_CANDrvFv                                                
0     00087b37  _Drv_CANEnable__12Class_CANDrvFUl                                                      
0     00087b40  _Drv_CANGlobalIntEnable__12Class_CANDrvFUlT1                                           
0     00087b4a  _Drv_CANGlobalIntDisable__12Class_CANDrvFUlT1                                          
0     00087b55  _Drv_CANMessageSet__12Class_CANDrvFUlT1P13tCANMsgObject11tMsgObjType                   
0     00087c46  _Drv_CANMessageGet__12Class_CANDrvFUlT1P13tCANMsgObjectb                               
0     00087d21  _Drv_CANDataRegWrite__12Class_CANDrvSFPUcPUli                                          
0     00087d3b  _Drv_CANIntStatus__12Class_CANDrvFUl13tCANIntStsReg                                    
0     00087d56  _Drv_CANStatusGet__12Class_CANDrvFUl10tCANStsReg                                       
0     00087d7f  _Drv_CANIntClear__12Class_CANDrvFUlT1                                                  
0     00087da6  _Drv_CANGlobalIntClear__12Class_CANDrvFUlT1                                            
0     00087db0  _Drv_CANDataRegRead__12Class_CANDrvSFPUcPUli                                           
0     00087dcb  _Drv_CANMsgObjCTLStatusGet__12Class_CANDrvFUlT1                                        
0     00087ded  _Drv_InitI2C__12Class_I2CDrvFv                                                         
0     00087e1a  _Drv_I2CRead__12Class_I2CDrvFUiiPUi                                                    
0     00087e6e  _Drv_I2CWordWrite__12Class_I2CDrvFUiT1                                                 
0     00087e90  _Drv_I2CPageWrite__12Class_I2CDrvFUiiPUi                                               
0     00087ec5  _Drv_I2CWriteAll__12Class_I2CDrvFPUiPiT1                                               
0     00087f3a  _Drv_InitADC__12Class_ADCDrvFv                                                         
0     0008806e  _Drv_AdcSetMode__12Class_ADCDrvFUiN21                                                  
0     000880f1  _Drv_CalAdcINL__12Class_ADCDrvFUi                                                      
0     0008811f  _Drv_InitPWM__12Class_PWMDrvFv                                                         
0     00088325  _Drv_InitCAP__12Class_CAPDrvFv                                                         
0     0008838f  _Drv_SysCtrlInit__12Class_SysDrvFv                                                     
0     000883ca  _Drv_InitPeripherals__12Class_SysDrvFv                                                 
0     000883fa  _Drv_InitSysPll__12Class_SysDrvFUiN31                                                  
0     0008847e  _Drv_SysIntOsc1Sel__12Class_SysDrvFv                                                   
0     0008848b  _Drv_SysIntOsc2Sel__12Class_SysDrvFv                                                   
0     00088498  _Drv_SysXtalOscSel__12Class_SysDrvFv                                                   
0     000884a7  _Drv_InitPeripheralClocks__12Class_SysDrvFv                                            
0     00088532  _Drv_InitPieCtrl__12Class_SysDrvFv                                                     
0     00088556  _Drv_InitPieVectTable__12Class_SysDrvFv                                                
0     0008857d  _Drv_InitCpuTimers__12Class_SysDrvFv                                                   
0     0008858f  _Drv_Int_InterruptFlagClear__12Class_SysDrvFv                                          
0     00088593  _Drv_InitPIE__12Class_SysDrvFv                                                         
0     000885a3  _Drv_InitInterrupts__12Class_SysDrvFv                                                  
0     000885b1  _Drv_DisableDog__17Class_WatchDogDrvFv                                                 
0     000885c0  _Drv_EnableDog__17Class_WatchDogDrvFv                                                  
0     000885cb  _Drv_KickDog__17Class_WatchDogDrvFv                                                    
0     000885dc  _Drv_Init__12Class_RAMDrvFv                                                            
0     000885ea  _Drv_RamCheck__12Class_RAMDrvFv                                                        
0     000886a9  _Drv_MemCopy__12Class_RAMDrvFPUiN21                                                    
0     000886c6  _Drv_CLAMemCopy__12Class_RAMDrvFPUlN21                                                 
0     000886d9  _Drv_SysTimer__14Class_TimerDrvFv                                                      
0     00088758  _Drv_usDelay__14Class_TimerDrvFl                                                       
0     00088771  _Drv_InitCMPSS__14Class_CMPSSDrvFv                                                     
0     0008879b  _App_InvAlgVarInit__23Class_InverterAlgorithmFv                                        
0     0008881c  _App_InvAlgParamConfig1__23Class_InverterAlgorithmFv                                   
0     00088b9d  _App_InvAlgParamConfig2__23Class_InverterAlgorithmFv                                   
0     00088e8b  _App_SysVarInit__12Class_SystemFv                                                      
0     00089053  _App_SysInitSunStreaker_208__12Class_SystemFv                                          
0     00089234  _App_SysInitSunStreaker_400__12Class_SystemFv                                          
0     00089415  _App_SysInitBasedUPSName__12Class_SystemFv                                             
0     0008952d  _App_ModuleOnline__12Class_SystemFv                                                    
0     0008955c  _App_SysParamConfig__12Class_SystemFv                                                  
0     0008971c  _App_DSPCheck__12Class_SystemFv                                                        
0     00089753  _App_FPGA_Ver__12Class_SystemFv                                                        
0     00089776  _App_Module_Ok__12Class_SystemFv                                                       
0     000897dc  _App_Module_LED__12Class_SystemFv                                                      
0     000898bf  _Alg_SysFault__12Class_SystemFv                                                        
0     00089965  _Alg_OperFault__12Class_SystemFv                                                       
0     000899a9  _App_IntelligentParall__12Class_SystemFv                                               
0     00089a10  _App_ModuleRelax_Affirm__12Class_SystemFv                                              
0     00089b00  _App_Relax_Command__12Class_SystemFv                                                   
0     00089c90  _App_FanNeedHighSpeed__12Class_SystemFv                                                
0     00089d00  _Alg_HeatFault__12Class_SystemFv                                                       
0     00089d59  _App_LimitPulseByPulseSet__12Class_SystemFv                                            
0     00089d7f  _APP_ModulePWMMicroAdj__12Class_SystemFv                                               
0     00089fb4  _App_FwupdateCondition__12Class_SystemFv                                               
0     00089fe0  _APP_EcoInvBpStatusF__12Class_SystemFv                                                 
0     0008a028  _App_PowCANInit__21Class_PowCANSchedulerFv                                             
0     0008a103  _Dat_Can_NoyBypCalculation__21Class_PowCANSchedulerFv                                  
0     0008a3ea  _App_PowCANConfigUpdate__21Class_PowCANSchedulerFv                                     
0     0008a451  _App_DigitalIOVarInit__15Class_DigitalIOFv                                             
0     0008a46d  _Dat_DigitalInput__15Class_DigitalIOFv                                                 
0     0008a9c3  _Dat_DigitalOutput__15Class_DigitalIOFv                                                
0     0008a9fc  _Dat_ServiceAndModuleTypeCheck__15Class_DigitalIOFv                                    
0     0008aa63  _App_IMCCtrl__15Class_DigitalIOFv                                                      
0     0008aa7f  _Dat_InvIDOk__15Class_DigitalIOFv                                                      
0     0008aa87  _Dat_BoardTypeCheck__15Class_DigitalIOFv                                               
0     0008ab53  _Dat_ModuleIDGet__15Class_DigitalIOFv                                                  
0     0008ac10  _Dat_FPGAIDCheck__15Class_DigitalIOFv                                                  
0     0008ac3f  _Dat_BreakerStatus__14Class_SwitchesFv                                                 
0     0008ad32  _Alg_INVKMFastChk__14Class_SwitchesFv                                                  
0     0008ae39  _Alg_STSShortFault__14Class_SwitchesFv                                                 
0     0008b09b  _Alg_STSOpenFault__14Class_SwitchesFv                                                  
0     0008b19a  _App_BpVarInit__12Class_BypassFv                                                       
0     0008b203  _App_BpParamConfig__12Class_BypassFv                                                   
0     0008b437  _Dat_BpRMS__12Class_BypassFv                                                           
0     0008b5cb  _Dat_VbpFlag__12Class_BypassFv                                                         
0     0008be70  _Alg_BpSeqFault__12Class_BypassFv                                                      
0     0008becb  _Alg_BpFault__12Class_BypassFv                                                         
0     0008bf61  _Dat_ECOBpFlag__12Class_BypassFv                                                       
0     0008bfc6  _App_InvVarInit__14Class_InverterFv                                                    
0     0008c052  _App_InvParamConfig__14Class_InverterFv                                                
0     0008c270  _Dat_VinvRMS__14Class_InverterFv                                                       
0     0008c3ef  _Dat_IinvRMS__14Class_InverterFv                                                       
0     0008c52c  _Dat_TempPowerGrant__14Class_InverterFv                                                
0     0008c5dc  _Dat_PinvRMS__14Class_InverterFv                                                       
0     0008c769  _Dat_VinvFlag__14Class_InverterFv                                                      
0     0008c97f  _Alg_InvFault__14Class_InverterFv                                                      
0     0008c9e7  _Alg_InvOverCurrentChk__14Class_InverterFv                                             
0     0008ca7d  _Alg_VoutToGnd_Fault__14Class_InverterFv                                               
0     0008cac9  _App_OutVarInit__12Class_OutputFv                                                      
0     0008cb16  _App_OutParamConfig__12Class_OutputFv                                                  
0     0008cb80  _Dat_VoutRMS__12Class_OutputFv                                                         
0     0008ccc4  _Dat_PoutRMS__12Class_OutputFv                                                         
0     0008ceaa  _Alg_VoutAbnormal__12Class_OutputFv                                                    
0     0008cf37  _Alg_ParaStatus__14Class_ParallelFv                                                    
0     0008cfd1  _Alg_ParaFault__14Class_ParallelFv                                                     
0     0008cff7  _App_DCBusVarInit__11Class_DCBusFv                                                     
0     0008d00e  _App_DCBusParamConfig__11Class_DCBusFv                                                 
0     0008d04e  _Dat_DCBusRMS__11Class_DCBusFv                                                         
0     0008d06f  _Alg_DCBusFault__11Class_DCBusFv                                                       
0     0008d15a  _App_MonitorVarInit__22Class_MonitorInterfaceFv                                        
0     0008d58b  _App_MonitorDeal__22Class_MonitorInterfaceFv                                           
0     0008d5ab  _App_MonInterfaceWrite__22Class_MonitorInterfaceFv                                     
0     0008db82  _App_MonitorOrder__22Class_MonitorInterfaceFv                                          
0     0008ddd2  _App_SendtoMonitor__22Class_MonitorInterfaceFv                                         
0     0008df26  _App_MonitorParam__22Class_MonitorInterfaceFv                                          
0     0008df9a  _App_MonInterfaceRead__22Class_MonitorInterfaceFv                                      
0     0008e6a7  _App_ParallelLocalData__22Class_MonitorInterfaceFv                                     
0     0008e70f  _Dat_LoadDeal__10Class_LoadFv                                                          
0     0008e72f  _Dat_LoadGrant__10Class_LoadFv                                                         
0     0008e7af  _Alg_ShortCircuitDetect__10Class_LoadFv                                                
0     0008e805  _Dat_LoadFlag__10Class_LoadFv                                                          
0     0008ebda  _Dat_OvloadFlag__10Class_LoadFv                                                        
0     0008ec83  _App_OvloadDelay__10Class_LoadFv                                                       
0     0008edcd  _App_OvloadSignal__10Class_LoadFv                                                      
0     0008ee10  _App_InvCtrl__21Class_InverterControlFv                                                
0     0008ee30  _App_InvOffReason__21Class_InverterControlFv                                           
0     0008ee81  _App_InvOnoffAgent__21Class_InverterControlFv                                          
0     0008f030  _App_InvOnoffAction__21Class_InverterControlFv                                         
0     0008f13e  _App_InvMaster__21Class_InverterControlFv                                              
0     0008f276  _App_InvTrace__21Class_InverterControlFv                                               
0     0008f28d  _App_InvSoftstart__21Class_InverterControlFv                                           
0     0008f360  _App_InvStandby__21Class_InverterControlFv                                             
0     0008f415  _App_TraceSignal__21Class_InverterControlFv                                            
0     0008f45e  _App_TraceControl__21Class_InverterControlFv                                           
0     0008f573  _App_TraceJudge__21Class_InverterControlFv                                             
0     0008f648  _App_XferOut__14Class_TransferFv                                                       
0     0008f6cb  _App_XferCommand__14Class_TransferFv                                                   
0     0008fc1c  _App_XferProcess__14Class_TransferFv                                                   
0     0008ffea  _App_XferExecute__14Class_TransferFv                                                   
0     00090252  _Alg_LBSSignal__9Class_LBSFv                                                           
0     000902e4  _App_ServiceMode__13Class_ServiceFv                                                    
0     0009033d  _App_ECO__9Class_ECOFv                                                                 
0     00090343  _App_ECOInvToBpFlagDeal__9Class_ECOFv                                                  
0     000903af  _App_FaultRecordTaxsis__17Class_FaultRecordFv                                          
0     00090481  _App_FaultRecord__17Class_FaultRecordFv                                                
0     0009065d  _Dat_EEPROMInit__12Class_EEPROMFv                                                      
0     0009069c  _App_ParamEEPROMW__12Class_EEPROMFv                                                    
0     00090853  _App_FaultEEPROMW__12Class_EEPROMFv                                                    
0     000908e3  _App_FaultRead__12Class_EEPROMFv                                                       
0     00090905  _App_FaultReadTaskInit__12Class_EEPROMFi                                               
0     00090953  _App_ParamReadTaskInit__12Class_EEPROMFv                                               
0     00090984  _App_EEPROMRead__12Class_EEPROMFv                                                      
0     000909b9  _App_EEPROMWrite__12Class_EEPROMFv                                                     
0     00090a04  _App_DSPResetInfoWrite__12Class_EEPROMFv                                               
0     00090a9d  _App_EEPROMAction__12Class_EEPROMFv                                                    
0     00090ae4  _App_EEPROMVerify__12Class_EEPROMFPUiT1Ui                                              
0     00090b07  _App_SelfAgingAlgVarInit__24Class_SelfAgingAlgorithmFv                                 
0     00090b24  _App_SelfAgingAlgParamConfig__24Class_SelfAgingAlgorithmFv                             
0     00090be9  _App_SelfAgingTargetUpdate__24Class_SelfAgingAlgorithmFv                               
0     00090c30  _Alg_Int_SelfAging__24Class_SelfAgingAlgorithmFv                                       
0     00090c53  _Alg_Int_AgingSPWM__24Class_SelfAgingAlgorithmFv                                       
0     00090da3  _App_DebugVarInit__11Class_DebugFv                                                     
0     00090dde  _DebugComandHandle__11Class_DebugFv                                                    
0     00090f38  _DebugAckMessage__11Class_DebugFv                                                      
0     00090f77  _Drv_ConfigStart__16Class_FPGAConfigFv                                                 
0     00090f99  _App_FPGAConfigProcess__16Class_FPGAConfigFv                                           
0     000910d3  _App_FPGAConfigError__16Class_FPGAConfigFUi                                            
0     000910e5  _App_SciFlashMain__15Class_FPGAFlashFv                                                 
0     00091b5b  _App_SCIVarInit__15Class_FPGAFlashFv                                                   
0     00091bc0  _cal_sumcheck__15Class_FPGAFlashFPUiUi                                                 
0     00091be2  _wCRC__15Class_FPGAFlashFPUiUi                                                         
0     00091c13  _VarReset__15Class_FPGAFlashFv                                                         
0     00091c65  _SciFrameOverTime__15Class_FPGAFlashFv                                                 
0     00091ca6  _App_FPGAFlashMain_CAN__15Class_FPGAFlashFv                                            
0     00091f74  _CANDat_MBox_Read__15Class_FPGAFlashFv                                                 
0     00091f78  _CANDat_MBox_Send__15Class_FPGAFlashFUiT1                                              
0     00091f88  ___CPR75__ProtocolSubCmdIni__14ProtocolSubCmdFP14SysCanProtocolMJ37JFPv_i              
0     00091f9e  _Excute__14ProtocolSubCmdFPv                                                           
0     00091fc3  _AppSubCmdIni__9AppSubCmdFP9SysCanAppM9SysCanAppFPv_i                                  
0     00091fd9  _Excute__9AppSubCmdFPv                                                                 
0     00091ffe  _SysCanRecvQueueIni__15SysCanRecvQueueFv                                               
0     0009200a  _InsQueue__15SysCanRecvQueueF26CAN_PACKED_PROTOCOL_STRUCT                              
0     00092033  _DelQueue__15SysCanRecvQueueFv                                                         
0     0009204b  _FlagQueue__15SysCanRecvQueueFv                                                        
0     0009205d  _GetOldestNode__15SysCanRecvQueueFv                                                    
0     0009206b  _SysCanXmitQueueIni__15SysCanXmitQueueFv                                               
0     00092077  _InsQueue__15SysCanXmitQueueF26CAN_PACKED_PROTOCOL_STRUCT                              
0     000920a0  _DelQueue__15SysCanXmitQueueFv                                                         
0     000920b8  _FlagQueue__15SysCanXmitQueueFv                                                        
0     000920ca  _GetOldestNode__15SysCanXmitQueueFv                                                    
0     000920d8  _SysCanFragXmitQueueIni__19SysCanFragXmitQueueFv                                       
0     000920e4  _InsQueue__19SysCanFragXmitQueueF19can_msg_data_struct                                 
0     0009210d  _DelQueue__19SysCanFragXmitQueueFv                                                     
0     00092125  _FlagQueue__19SysCanFragXmitQueueFv                                                    
0     00092137  _GetOldestNode__19SysCanFragXmitQueueFv                                                
0     00092145  _SysCanProtocolIni__14SysCanProtocolFv                                                 
0     00092254  _SysCanRecvFcb__14SysCanProtocolFPv                                                    
0     0009229c  _SysCanXmitFcb__14SysCanProtocolFPv                                                    
0     000922d9  _XmitFramePost__14SysCanProtocolFP26CAN_PACKED_PROTOCOL_STRUCT                         
0     00092332  _MsgRecvProc__14SysCanProtocolFP19can_msg_data_struct                                  
0     00092392  _MsgXmitProc__14SysCanProtocolFP19can_msg_data_struct                                  
0     000923c7  _SetFragRecvOkHandleFcb__14SysCanProtocolFP11CommandBase                               
0     000923e3  _SetFragXmitErrHandleFcb__14SysCanProtocolFP11CommandBase                              
0     000923fd  _SetFragXmitOkHandleFcb__14SysCanProtocolFP11CommandBase                               
0     00092417  _Timer_Expire_Handle__14SysCanProtocolFv                                               
0     0009242e  _FrameParseToApdu__14SysCanProtocolFP19can_msg_data_structP26CAN_PACKED_PROTOCOL_STRUCT
0     0009249f  _FrameParseToPpdu__14SysCanProtocolFP26CAN_PACKED_PROTOCOL_STRUCTP19can_msg_data_struct
0     00092522  _FragMsgXmitStateMachineEnty__14SysCanProtocolFv                                       
0     0009255a  _FragMsgXmitStateMachine__14SysCanProtocolFP26CAN_PACKED_PROTOCOL_STRUCT               
0     00092750  _FragMsgRecvStateMachine__14SysCanProtocolFP26CAN_PACKED_PROTOCOL_STRUCT               
0     00092a05  _FragAckTimeoutFcb__14SysCanProtocolFv                                                 
0     00092a47  _FragXmitBusyTimeoutFcb__14SysCanProtocolFv                                            
0     00092a89  _CANFragRecvTimeoutFcb__14SysCanProtocolFv                                             
0     00092aa5  _Timer_Post__14SysCanProtocolFP14TIMER_HANDLE_T                                        
0     00092abb  _Timer_Flush__14SysCanProtocolFP14TIMER_HANDLE_T                                       
0     00092acc  _SysCanDataExchgIni__15SysCanDataExchgFv                                               
0     00092ae6  _InterfaceDataProc__15SysCanDataExchgFv                                                
0     00092d0c  _GetDataExchgPtr__15SysCanDataExchgSFv                                                 
0     00092d33  _GetStateCovMsg__15SysCanDataExchgFP19can_msg_data_struct                              
0     00092d6a  _StateCovMsgXmitState__15SysCanDataExchgFi                                             
0     00092d79  _StateXmitMsgGen__15SysCanDataExchgFUi                                                 
0     00092df4  _GetAlrmCovMsg__15SysCanDataExchgFP19can_msg_data_struct                               
0     00092e2c  _AlrmCovMsgXmitState__15SysCanDataExchgFi                                              
0     00092e3b  _AlrmXmitMsgGen__15SysCanDataExchgFUi                                                  
0     00092eb9  _GetEventLogMsg__15SysCanDataExchgFP19can_msg_data_struct                              
0     00092f35  _ReqSetMsg__15SysCanDataExchgFP19can_msg_data_struct                                   
0     00092f9b  _AlarmEventXmitMsgGen__15SysCanDataExchgFUi                                            
0     00093017  _StateEventXmitMsgGen__15SysCanDataExchgFUi                                            
0     00093090  _GetParallelStateMsg__15SysCanDataExchgFP19can_msg_data_struct                         
0     000930cb  _ParallelStateXmitMsgGen__15SysCanDataExchgFUi                                         
0     00093147  _SyncFlagDelayProc__15SysCanDataExchgFP19can_msg_data_struct                           
0     000931d5  _GetStateSyncMsg__15SysCanDataExchgFP19can_msg_data_struct                             
0     00093251  _StateSyncMsgXmitState__15SysCanDataExchgFi                                            
0     00093260  _GetAlrmSyncMsg__15SysCanDataExchgFP19can_msg_data_struct                              
0     000932ac  _AlrmSyncMsgXmitState__15SysCanDataExchgFi                                             
0     000932bb  _GetAnalogSyncMsg__15SysCanDataExchgFP19can_msg_data_struct                            
0     00093311  _AnalogSyncMsgXmitState__15SysCanDataExchgFi                                           
0     00093320  _PeriodAnalogSyncMsg__15SysCanDataExchgFP19can_msg_data_struct                         
0     00093386  _MonitorSyncMsgProc__15SysCanDataExchgFv                                               
0     000933ce  _CfgMsgRecvProc__15SysCanDataExchgFP19can_msg_data_struct                              
0     00093433  _StateMsgRecvProc__15SysCanDataExchgFP19can_msg_data_struct                            
0     00093471  _SyncMsgProc__15SysCanDataExchgFP19can_msg_data_struct                                 
0     000934c2  _CfgMsgFromMonProc__15SysCanDataExchgFP19can_msg_data_structUi                         
0     000935d3  _CfgMsgToMonProc__15SysCanDataExchgFP19can_msg_data_structUi                           
0     00093670  _SyncTimeMsgProc__15SysCanDataExchgFP19can_msg_data_struct                             
0     000936a1  _AlrmMsgRecvProc__15SysCanDataExchgFP19can_msg_data_struct                             
0     0009370c  _CtrlMsgRecvProc__15SysCanDataExchgFP19can_msg_data_struct                             
0     000938b4  _BattEodTurnOff__15SysCanDataExchgFv                                                   
0     000938c6  _BattTrip__15SysCanDataExchgFv                                                         
0     000938d8  _OutputEnableCmd__15SysCanDataExchgFv                                                  
0     000938ea  _OutputDisableCmd__15SysCanDataExchgFv                                                 
0     000938fc  _BattGndPtcCmd__15SysCanDataExchgFv                                                    
0     0009390e  _FaultClrCmd__15SysCanDataExchgFv                                                      
0     0009392e  _MaualStartupCmd__15SysCanDataExchgFv                                                  
0     00093954  _MaualShutCmd__15SysCanDataExchgFv                                                     
0     0009397a  _EpoCmd__15SysCanDataExchgFv                                                           
0     0009398c  _AbnormalShutConfirmCmd__15SysCanDataExchgFv                                           
0     0009399e  _AbnormalShutCancelCmd__15SysCanDataExchgFv                                            
0     000939b0  _IndirectSwitchCmd__15SysCanDataExchgFv                                                
0     000939c2  _RecFlashUpdate__15SysCanDataExchgFv                                                   
0     000939d8  _InvFlashUpdate__15SysCanDataExchgFv                                                   
0     00093a0c  _BypFlashUpdate__15SysCanDataExchgFv                                                   
0     00093a22  _RecFPGAFlashUpdate__15SysCanDataExchgFv                                               
0     00093a30  _InvFPGAFlashUpdate__15SysCanDataExchgFv                                               
0     00093a64  _BypFPGAFlashUpdate__15SysCanDataExchgFv                                               
0     00093a72  _FragXmitResult__15SysCanDataExchgFP19can_msg_data_structi                             
0     00093a84  _FragMsgPacked__15SysCanDataExchgFP19can_msg_data_struct                               
0     00093aa5  _CfgFragMsgPacked__15SysCanDataExchgFP19can_msg_data_struct                            
0     00093aed  _AnalogMsgRecvProc__15SysCanDataExchgFP19can_msg_data_struct                           
0     00093b34  _GetFaultData__15SysCanDataExchgFP19can_msg_data_struct                                
0     00093b6a  _AnalogRecvMsgObjsInit__15SysCanDataExchgFv                                            
0     00093b91  _CtrlMsgObjsInit__15SysCanDataExchgFv                                                  
0     00093bbd  _CovSyncMsgObjInit__15SysCanDataExchgFv                                                
0     00093cf3  _CfgMsgObjsInit__15SysCanDataExchgFv                                                   
0     00093d73  _AnalogXmitMsgGen__15SysCanDataExchgFUi                                                
0     00093def  _PeriodPowerXmitMsgGen__15SysCanDataExchgFUi                                           
0     0009400b  _CfgMsgRqPacked__15SysCanDataExchgFP19can_msg_data_structi                             
0     0009403a  _CfgMsgRsPacked__15SysCanDataExchgFP19can_msg_data_structi                             
0     0009408a  _GetResendSysSetFlag__15SysCanDataExchgFv                                              
0     000940a8  _RestartResendTimer__15SysCanDataExchgFv                                               
0     000940b8  _EndResendTimer__15SysCanDataExchgFv                                                   
0     000940c9  _GenStateEvent__15SysCanDataExchgFv                                                    
0     000942a0  _GenAlarmEvent__15SysCanDataExchgFv                                                    
0     00094565  _FaultFragMsgPacked__15SysCanDataExchgFP19can_msg_data_struct                          
0     0009458e  _ParallelMsgRecvProc__15SysCanDataExchgFP19can_msg_data_struct                         
0     000945b5  _MaintParallelData__15SysCanDataExchgFv                                                
0     0009462d  _BypMaintMsgRecvProc__15SysCanDataExchgFP19can_msg_data_struct                         
0     00094650  _RackStateMsgRecvProc__15SysCanDataExchgFP19can_msg_data_struct                        
0     00094679  _GetSyncMonitorCnt__15SysCanDataExchgFv                                                
0     000946a9  _MonRealMsgRecvProc__15SysCanDataExchgFP19can_msg_data_struct                          
0     000946cc  _MonitorCanErrDetect__15SysCanDataExchgFv                                              
0     00094711  _MsgRecvProc__9SysCanAppFv                                                             
0     0009473c  _MainRoutie__9SysCanAppFv                                                              
0     0009475a  _SysCanInitial__9SysCanAppFv                                                           
0     000947af  _CovMsgProc__9SysCanAppFv                                                              
0     0009483a  _SyncMsgProc__9SysCanAppFv                                                             
0     000948d6  _FaultDataXimt__9SysCanAppFv                                                           
0     0009490c  _RecvMsgDispatch__9SysCanAppFP19can_msg_data_struct                                    
0     00094976  _FragMsgPost__9SysCanAppFv                                                             
0     000949a5  _FragXmitOkHandle__9SysCanAppFPv                                                       
0     000949be  _FragXmitErrHandle__9SysCanAppFPv                                                      
0     000949d4  _FragRecvOkHandle__9SysCanAppFPv                                                       
0     000949e4  _Excute__30TemplateCmd__tm__11_9SysCanAppFPv_i                                         
0     00094a09  ___sti___17_MainProcedure_cpp_6cdd801d                                                 
0     00094a12  _PIE_RESERVED__Fv                                                                      
0     00094a55  _TIMER1_ISR                                                                            
0     00094a5a  _TIMER2_ISR                                                                            
0     00094a5f  _DATALOG_ISR                                                                           
0     00094a64  _RTOS_ISR                                                                              
0     00094a69  _EMU_ISR                                                                               
0     00094a6e  _NMI_ISR                                                                               
0     00094a73  _ILLEGAL_ISR                                                                           
0     00094a78  _USER1_ISR                                                                             
0     00094a7d  _USER2_ISR                                                                             
0     00094a82  _USER3_ISR                                                                             
0     00094a87  _USER4_ISR                                                                             
0     00094a8c  _USER5_ISR                                                                             
0     00094a91  _USER6_ISR                                                                             
0     00094a96  _USER7_ISR                                                                             
0     00094a9b  _USER8_ISR                                                                             
0     00094aa0  _USER9_ISR                                                                             
0     00094aa5  _USER10_ISR                                                                            
0     00094aaa  _USER11_ISR                                                                            
0     00094aaf  _USER12_ISR                                                                            
0     00094ab4  _ADCA1_ISR                                                                             
0     00094ab9  _ADCB1_ISR                                                                             
0     00094abe  _XINT1_ISR                                                                             
0     00094ac3  _XINT2_ISR                                                                             
0     00094ac8  _ADCD1_ISR                                                                             
0     00094acd  _TIMER0_ISR                                                                            
0     00094ad2  _WAKE_ISR                                                                              
0     00094ad7  _EPWM1_TZ_ISR                                                                          
0     00094adc  _EPWM2_TZ_ISR                                                                          
0     00094ae1  _EPWM3_TZ_ISR                                                                          
0     00094ae6  _EPWM4_TZ_ISR                                                                          
0     00094aeb  _EPWM5_TZ_ISR                                                                          
0     00094af0  _EPWM6_TZ_ISR                                                                          
0     00094af5  _EPWM7_TZ_ISR                                                                          
0     00094afa  _EPWM8_TZ_ISR                                                                          
0     00094aff  _EPWM1_ISR                                                                             
0     00094b04  _EPWM2_ISR                                                                             
0     00094b09  _EPWM3_ISR                                                                             
0     00094b0e  _EPWM4_ISR                                                                             
0     00094b13  _EPWM5_ISR                                                                             
0     00094b18  _EPWM6_ISR                                                                             
0     00094b1d  _EPWM7_ISR                                                                             
0     00094b22  _EPWM8_ISR                                                                             
0     00094b27  _ECAP1_ISR                                                                             
0     00094b2c  _ECAP2_ISR                                                                             
0     00094b31  _ECAP3_ISR                                                                             
0     00094b36  _ECAP4_ISR                                                                             
0     00094b3b  _ECAP5_ISR                                                                             
0     00094b40  _ECAP6_ISR                                                                             
0     00094b45  _EQEP1_ISR                                                                             
0     00094b4a  _EQEP2_ISR                                                                             
0     00094b4f  _EQEP3_ISR                                                                             
0     00094b54  _SPIA_RX_ISR                                                                           
0     00094b59  _SPIA_TX_ISR                                                                           
0     00094b5e  _SPIB_RX_ISR                                                                           
0     00094b63  _SPIB_TX_ISR                                                                           
0     00094b68  _MCBSPA_RX_ISR                                                                         
0     00094b6d  _MCBSPA_TX_ISR                                                                         
0     00094b72  _MCBSPB_RX_ISR                                                                         
0     00094b77  _MCBSPB_TX_ISR                                                                         
0     00094b7c  _DMA_CH1_ISR                                                                           
0     00094b81  _DMA_CH2_ISR                                                                           
0     00094b86  _DMA_CH3_ISR                                                                           
0     00094b8b  _DMA_CH4_ISR                                                                           
0     00094b90  _DMA_CH5_ISR                                                                           
0     00094b95  _DMA_CH6_ISR                                                                           
0     00094b9a  _I2CA_ISR                                                                              
0     00094b9f  _I2CA_FIFO_ISR                                                                         
0     00094ba4  _I2CB_ISR                                                                              
0     00094ba9  _I2CB_FIFO_ISR                                                                         
0     00094bae  _SCIC_RX_ISR                                                                           
0     00094bb3  _SCIC_TX_ISR                                                                           
0     00094bb8  _SCID_RX_ISR                                                                           
0     00094bbd  _SCID_TX_ISR                                                                           
0     00094bc2  _SCIA_RX_ISR                                                                           
0     00094bc7  _SCIA_TX_ISR                                                                           
0     00094bcc  _SCIB_RX_ISR                                                                           
0     00094bd1  _SCIB_TX_ISR                                                                           
0     00094bd6  _CANA0_ISR                                                                             
0     00094bdb  _CANA1_ISR                                                                             
0     00094be0  _CANB0_ISR                                                                             
0     00094be5  _CANB1_ISR                                                                             
0     00094bea  _ADCA_EVT_ISR                                                                          
0     00094bef  _ADCA2_ISR                                                                             
0     00094bf4  _ADCA3_ISR                                                                             
0     00094bf9  _ADCA4_ISR                                                                             
0     00094bfe  _ADCB_EVT_ISR                                                                          
0     00094c03  _ADCB2_ISR                                                                             
0     00094c08  _ADCB3_ISR                                                                             
0     00094c0d  _ADCB4_ISR                                                                             
0     00094c12  _CLA1_1_ISR                                                                            
0     00094c17  _CLA1_2_ISR                                                                            
0     00094c1c  _CLA1_3_ISR                                                                            
0     00094c21  _CLA1_4_ISR                                                                            
0     00094c26  _CLA1_5_ISR                                                                            
0     00094c2b  _CLA1_6_ISR                                                                            
0     00094c30  _CLA1_7_ISR                                                                            
0     00094c35  _CLA1_8_ISR                                                                            
0     00094c3a  _XINT3_ISR                                                                             
0     00094c3f  _XINT4_ISR                                                                             
0     00094c44  _XINT5_ISR                                                                             
0     00094c49  _VCU_ISR                                                                               
0     00094c4e  _FPU_OVERFLOW_ISR                                                                      
0     00094c53  _FPU_UNDERFLOW_ISR                                                                     
0     00094c58  _IPC0_ISR                                                                              
0     00094c5d  _IPC1_ISR                                                                              
0     00094c62  _IPC2_ISR                                                                              
0     00094c67  _IPC3_ISR                                                                              
0     00094c6c  _EPWM9_TZ_ISR                                                                          
0     00094c71  _EPWM10_TZ_ISR                                                                         
0     00094c76  _EPWM11_TZ_ISR                                                                         
0     00094c7b  _EPWM12_TZ_ISR                                                                         
0     00094c80  _EPWM9_ISR                                                                             
0     00094c85  _EPWM10_ISR                                                                            
0     00094c8a  _EPWM11_ISR                                                                            
0     00094c8f  _EPWM12_ISR                                                                            
0     00094c94  _SD1_ISR                                                                               
0     00094c99  _SD2_ISR                                                                               
0     00094c9e  _SPIC_RX_ISR                                                                           
0     00094ca3  _SPIC_TX_ISR                                                                           
0     00094ca8  _USBA_ISR                                                                              
0     00094cad  _ADCD_EVT_ISR                                                                          
0     00094cb2  _ADCD2_ISR                                                                             
0     00094cb7  _ADCD3_ISR                                                                             
0     00094cbc  _ADCD4_ISR                                                                             
0     00094cc1  _EMIF_ERROR_ISR                                                                        
0     00094cc6  _RAM_CORRECTABLE_ERROR_ISR                                                             
0     00094ccb  _FLASH_CORRECTABLE_ERROR_ISR                                                           
0     00094cd0  _RAM_ACCESS_VIOLATION_ISR                                                              
0     00094cd5  _SYS_PLL_SLIP_ISR                                                                      
0     00094cda  _AUX_PLL_SLIP_ISR                                                                      
0     00094cdf  _CLA_OVERFLOW_ISR                                                                      
0     00094ce4  _CLA_UNDERFLOW_ISR                                                                     
0     00094ce9  _PIE_RESERVED_ISR                                                                      
0     00094cee  _EMPTY_ISR                                                                             
0     00094cf3  _NOTUSED_ISR                                                                           
0     00094cf8  _ECAN0INTA_ISR__Fv                                                                     
0     00094db1  _cla1Isr1__Fv                                                                          
0     00094dbe  _cla1Isr2__Fv                                                                          
0     00094dc4  _cla1Isr3__Fv                                                                          
0     00094dca  _cla1Isr4__Fv                                                                          
0     00094dd0  _cla1Isr5__Fv                                                                          
0     00094dd6  _cla1Isr6__Fv                                                                          
0     00094ddc  _cla1Isr7__Fv                                                                          
0     00094de2  _cla1Isr8__Fv                                                                          
0     00094deb  _free                                                                                  
0     00094e31  _minit                                                                                 
0     00094e54  _malloc                                                                                
0     00094eb1  _realloc                                                                               
0     00094f65  _max_free                                                                              
0     00094f84  _free_memory                                                                           
0     00094f9f  _chkheap                                                                               
0     00094fa1  _calloc                                                                                
0     00094fb8  LL$$DIV                                                                                
0     00094ff4  LL$$MOD                                                                                
0     0009502e  ULL$$DIV                                                                               
0     0009505d  ULL$$MOD                                                                               
0     000950bf  FS$$DIV                                                                                
0     00095142  FS$$MPY                                                                                
0     0009519c  _c_int00                                                                               
0     000951f0  L$$DIV                                                                                 
0     000951ff  L$$MOD                                                                                 
0     0009520d  UL$$DIV                                                                                
0     00095214  UL$$MOD                                                                                
0     0009521a  C$$EXIT                                                                                
0     0009521a  _abort                                                                                 
0     0009521c  _exit                                                                                  
0     00095243  FS$$TOI                                                                                
0     00095282  ___add_dtor                                                                            
0     0009528d  _copy_in                                                                               
0     000952b1  I$$DIV                                                                                 
0     000952c2  I$$MOD                                                                                 
0     000952d3  ___nw__FUl                                                                             
0     000952f3  _memcpy                                                                                
0     00095310  I$$TOFS                                                                                
0     0009532a  __args_main                                                                            
0     00095343  LL$$MPY                                                                                
0     00095357  _memset                                                                                
0     00095363  U$$DIV                                                                                 
0     00095368  U$$MOD                                                                                 
0     0009536e  __register_unlock                                                                      
0     00095372  __register_lock                                                                        
0     00095376  __nop                                                                                  
0     0009537f  ___dl__FPv                                                                             
0     00095384  ___pure_virtual_called                                                                 
0     00095388  ___abort_execution                                                                     
0     0009538b  __system_pre_init                                                                      
0     0009538d  ___default_new_handler__Fv                                                             
0     0009538e  __system_post_cinit                                                                    
0     0009538f  ___etext__                                                                             
0     0009538f  etext                                                                                  
0     00095390  _RamfuncsLoadStart                                                                     
0     000953b8  _RamfuncsLoadEnd                                                                       
0     00097402  ___vtbl__14ProtocolSubCmd                                                              
0     0009740e  ___vtbl__30TemplateCmd__tm__11_9SysCanApp                                              
0     00097449  _CriticalIntFuncsSecuredLoadStart                                                      
0     00097a22  _CriticalIntFuncsSecuredLoadEnd                                                        
0     00097a24  ___cinit__                                                                             
0     00097a24  cinit                                                                                  
0     00097abc  ___pinit__                                                                             
0     00097abc  pinit                                                                                  
1     00000400  __stack                                                                                
1     00000600  __STACK_END                                                                            
1     00000b00  _AdcaResultRegs                                                                        
1     00000b20  _AdcbResultRegs                                                                        
1     00000b60  _AdcdResultRegs                                                                        
1     00000c00  _CpuTimer0Regs                                                                         
1     00000c08  _CpuTimer1Regs                                                                         
1     00000c10  _CpuTimer2Regs                                                                         
1     00000ce0  _PieCtrlRegs                                                                           
1     00000d00  _EmuKey                                                                                
1     00000d00  _PieVectTable                                                                          
1     00000d01  _EmuBMode                                                                              
1     00001000  _DmaRegs                                                                               
1     00001400  _Cla1Regs                                                                              
1     00004000  _EPwm1Regs                                                                             
1     00004100  _EPwm2Regs                                                                             
1     00004200  _EPwm3Regs                                                                             
1     00004300  _EPwm4Regs                                                                             
1     00004400  _EPwm5Regs                                                                             
1     00004500  _EPwm6Regs                                                                             
1     00004600  _EPwm7Regs                                                                             
1     00004700  _EPwm8Regs                                                                             
1     00004800  _EPwm9Regs                                                                             
1     00004900  _EPwm10Regs                                                                            
1     00004a00  _EPwm11Regs                                                                            
1     00004b00  _EPwm12Regs                                                                            
1     00005000  _ECap1Regs                                                                             
1     00005020  _ECap2Regs                                                                             
1     00005040  _ECap3Regs                                                                             
1     00005060  _ECap4Regs                                                                             
1     00005080  _ECap5Regs                                                                             
1     000050a0  _ECap6Regs                                                                             
1     00005100  _EQep1Regs                                                                             
1     00005140  _EQep2Regs                                                                             
1     00005180  _EQep3Regs                                                                             
1     00005c00  _DacaRegs                                                                              
1     00005c10  _DacbRegs                                                                              
1     00005c20  _DaccRegs                                                                              
1     00005c80  _Cmpss1Regs                                                                            
1     00005ca0  _Cmpss2Regs                                                                            
1     00005cc0  _Cmpss3Regs                                                                            
1     00005ce0  _Cmpss4Regs                                                                            
1     00005d00  _Cmpss5Regs                                                                            
1     00005d20  _Cmpss6Regs                                                                            
1     00005d40  _Cmpss7Regs                                                                            
1     00005d60  _Cmpss8Regs                                                                            
1     00005e00  _Sdfm1Regs                                                                             
1     00005e80  _Sdfm2Regs                                                                             
1     00006000  _McbspaRegs                                                                            
1     00006040  _McbspbRegs                                                                            
1     00006100  _SpiaRegs                                                                              
1     00006110  _SpibRegs                                                                              
1     00006120  _SpicRegs                                                                              
1     00007000  _WdRegs                                                                                
1     00007060  _NmiIntruptRegs                                                                        
1     00007070  _XintRegs                                                                              
1     00007200  _SciaRegs                                                                              
1     00007210  _ScibRegs                                                                              
1     00007220  _ScicRegs                                                                              
1     00007230  _ScidRegs                                                                              
1     00007300  _I2caRegs                                                                              
1     00007340  _I2cbRegs                                                                              
1     00007400  _AdcaRegs                                                                              
1     00007480  _AdcbRegs                                                                              
1     00007580  _AdcdRegs                                                                              
1     00007900  _InputXbarRegs                                                                         
1     00007920  _XbarRegs                                                                              
1     00007940  _SyncSocRegs                                                                           
1     00007980  _DmaClaSrcSelRegs                                                                      
1     00007a00  _EPwmXbarRegs                                                                          
1     00007a80  _OutputXbarRegs                                                                        
1     00007c00  _GpioCtrlRegs                                                                          
1     00007f00  _GpioDataRegs                                                                          
1     0000c000  _objRAMDrv                                                                             
1     0000c001  _objPWMDrv                                                                             
1     0000c002  _objSCIDrv                                                                             
1     0000c003  _objCMPSSDrv                                                                           
1     0000c004  _objWatchDogDrv                                                                        
1     0000c005  _objCLA                                                                                
1     0000c006  _objCANDrv                                                                             
1     0000c007  _objI2CDrv                                                                             
1     0000c008  _objFlashDrv                                                                           
1     0000c009  _objCAPDrv                                                                             
1     0000c00a  _objGPIODrv                                                                            
1     0000c00b  _g_u16_INTRunTime                                                                      
1     0000c00c  _g_u16_MainRunTimeMax                                                                  
1     0000c00d  _g_u16_INTRunTimeMax                                                                   
1     0000c00e  _g_i16_IntCnt1Per4_0                                                                   
1     0000c00f  _g_i16_IntCnt1Per2_0                                                                   
1     0000c010  _objPowCANPro                                                                          
1     0000c011  _objFlashUpdate                                                                        
1     0000c012  _objECO                                                                                
1     0000c013  _g_u16_MainRunTime                                                                     
1     0000c014  _u16_FPGA_Flash_CANInit                                                                
1     0000c015  _objService                                                                            
1     0000c017  _objSysDrv                                                                             
1     0000c01a  _pCanIsrXmitFcb                                                                        
1     0000c01c  _m_pDataExchgPtr__15SysCanDataExchg                                                    
1     0000c01e  _pCanIsrRecvFcb                                                                        
1     0000c020  _g_ulRxMsgCount                                                                        
1     0000c022  _g_bErrFlag                                                                            
1     0000c024  _g_ulTxMsgCount                                                                        
1     0000c026  _objFaultRecord                                                                        
1     0000c02a  _objFPGAConfig                                                                         
1     0000c034  _ReceiveFrame                                                                          
1     0000c040  _objParallel                                                                           
1     0000c047  _ucRXAMsgData                                                                          
1     0000c04f  _ucTXAMsgData                                                                          
1     0000c057  _ucRXBMsgData                                                                          
1     0000c05f  _ucTXBMsgData                                                                          
1     0000c067  _objTimerDrv                                                                           
1     0000c070  _sTXCANAMessage                                                                        
1     0000c080  _sRXCANBMessage                                                                        
1     0000c08a  _sRXCANAMessage                                                                        
1     0000c094  _sTXCANBMessage                                                                        
1     0000c09e  _objLBS                                                                                
1     0000c0ac  _objDCBus                                                                              
1     0000c0c0  _objSwitches                                                                           
1     0000c0cf  _objInvCtrl                                                                            
1     0000c0de  _uInvAnalogLen                                                                         
1     0000c100  _objSPIDrv                                                                             
1     0000c140  _objXfer                                                                               
1     0000c180  _objEEPROM                                                                             
1     0000c1c0  _objADCDrv                                                                             
1     0000c200  _objLoad                                                                               
1     0000c240  _objSelfAgingAlg                                                                       
1     0000c280  _objDebug                                                                              
1     0000c2c0  _objDigitalIO                                                                          
1     0000c340  _objBypass                                                                             
1     0000c3c0  _objOutput                                                                             
1     0000c480  _objInvAlg                                                                             
1     0000c540  _objSystem                                                                             
1     0000c600  _objMonInterface                                                                       
1     0000c700  _objSysCanApp                                                                          
1     0000c840  _objFPGAFlash                                                                          
1     0000ca40  _objPowCANSched                                                                        
1     0000cc80  _objProtocol                                                                           
1     0000cf80  _objDataExchg                                                                          
1     0000d340  _objInverter                                                                           
1     0000d9b6  ___TI_enable_exit_profile_output                                                       
1     0000d9b8  ___TI_cleanup_ptr                                                                      
1     0000d9ba  ___TI_dtors_ptr                                                                        
1     0000d9bc  __lock                                                                                 
1     0000d9be  __unlock                                                                               
1     0000d9c1  ___atexit_func_id__                                                                    
1     0000dac2  __new_handler                                                                          
1     0000e800  __sys_memory                                                                           
1     00012000  _DebugRxBuff                                                                           
1     00012000  _FPGACodeEEPROMBuff                                                                    
1     00012000  _uFaultRecord                                                                          
1     00012080  _u16FaultRecordRead                                                                    
1     000120c0  _byCRCLoArrayFlash                                                                     
1     00012100  _uFaultRecordBuff                                                                      
1     000121c0  _byCRCHiArrayFlash                                                                     
1     000122c0  _m_u16_SCIRxBuff                                                                       
1     00012400  _FlashBuffer                                                                           
1     00012800  _st_FlashVariable                                                                      
1     00012f00  _DebugEEPROMBuff                                                                       
1     00047000  _Emif1Regs                                                                             
1     0005d000  _DevCfgRegs                                                                            
1     0005d180  _AnalogSubsysRegs                                                                      
1     0005d200  _ClkCfgRegs                                                                            
1     0005d300  _CpuSysRegs                                                                            
1     0005e608  _RomPrefetchRegs                                                                       
1     0005f000  _DcsmZ1Regs                                                                            
1     0005f040  _DcsmZ2Regs                                                                            
1     0005f070  _DcsmCommonRegs                                                                        
1     0005f400  _MemCfgRegs                                                                            
1     0005f480  _Emif1ConfigRegs                                                                       
1     0005f4c0  _AccessProtectionRegs                                                                  
1     0005f500  _MemoryErrorRegs                                                                       
1     0005f540  _RomWaitStateRegs                                                                      
1     0005f800  _Flash0CtrlRegs                                                                        
1     0005fb00  _Flash0EccRegs                                                                         
1     00078000  _DcsmZ1Otp                                                                             
1     00078200  _DcsmZ2Otp                                                                             
abs   00000000  _Cla1ConstLoadSize                                                                     
abs   00000000  _Cla1funcsLoadSize                                                                     
abs   00000028  _RamfuncsLoadSize                                                                      
abs   00000028  _RamfuncsRunSize                                                                       
abs   00000100  CLA_SCRATCHPAD_SIZE                                                                    
abs   00000200  __STACK_SIZE                                                                           
abs   00000400  __SYSMEM_SIZE                                                                          
abs   ffffffff  ___TI_pprof_out_hndl                                                                   
abs   ffffffff  ___TI_prof_data_size                                                                   
abs   ffffffff  ___TI_prof_data_start                                                                  
abs   ffffffff  ___binit__                                                                             
abs   ffffffff  ___c_args__                                                                            
abs   ffffffff  binit                                                                                  

[803 symbols]
